:1000000000000220757200009D7200009F720000C7
:10001000A1720000A3720000A572000000000000A1
:10002000000000000000000000000000A7720000B7
:10003000A972000000000000AB720000AD72000069
:10004000AF720000855100001D770000A171000013
:10005000AD710000AF720000AF720000AF7200001F
:10006000AF720000AF72000041330000AF720000B9
:10007000AF720000AF720000AF720000AF720000FC
:10008000AF720000A1770000AF720000AF720000F5
:10009000AF720000AF720000AF720000AF720000DC
:1000A000AF720000AF720000AF720000AF720000CC
:1000B000AF720000AF7200000000000000000000FE
:1000C000AF720000AF720000AF720000AF720000AC
:1000D000AF720000AF720000AF72000000000000BD
:1000E0000000000000000000000000000000000010
:1000F0000000000000000000000000000000000000
:1001000000000000000000000000000000000000EF
:1001100000000000000000000000000000000000DF
:1004000010B5054C237833B9044B13B10448AFF34E
:1004100000800123237010BD340200200000000082
:1004200078CB000008B5034B1BB103490348AFF379
:10043000008008BD000000003802002078CB0000DA
:10044000154B002B08BF134B9D46A3F5803A0021A6
:100450008B460F461348144A121A09F039FC0F4B09
:10046000002B00D098470E4B002B00D0984700205F
:10047000002104000D000D48002802D00C48AFF305
:10048000008009F0DDFB2000290007F09FF909F04A
:10049000B1FB00BF000008000000022000000000C7
:1004A0000000000034020020F88D01200000000050
:1004B0000000000010F0010310D104280CD90368DB
:1004C000C3F30F1343B1013B9B001A1DC1180979F7
:1004D00011B101339342F9D1184670470023FBE76D
:1004E000037883B11A0601D40130704703F0C003CA
:1004F000C02B08BF0130024610460132037803F0DA
:10050000C003802BF8D0704708B5002103780BB9E1
:10051000084608BDFFF7E4FF0131F7E738B50022D0
:1005200004460D46411C092003F016FA40B1630051
:10053000024643F0010342F8043F0023A34200DBDC
:1005400038BD55F8231042F8041F0133F6E701289F
:1005500038B504DC1C20BDE8384000F0FBBF0D6856
:10056000EA0701D41120F6E74868C30706D4042837
:1005700004D9036803F00F03042B01D00E20EAE72F
:1005800003F04EF86D10002D044603DDFFF7BCFFAD
:10059000A84206DA1220DEE72046FFF7A1FF013D60
:1005A0000446012DF8D120787F2808DDDF280ADCF9
:1005B0006378800100F4F86003F03F0318434000C3
:1005C00040F0010038BDEF280ADC637800039B018E
:1005D00080B203F47C630343A07800F03F00EDE7B2
:1005E000F72810DC637880041B0303F47C3300F4E9
:1005F000E0101843E37803F03F030343A078800141
:1006000000F47C60DAE74FF0FF30D8E7486838B58F
:10061000C3070D4606D4042804D9036803F00F026B
:10062000092A04D00B20BDE8384000F093BF44688D
:10063000C3F30F1364105A1EA2420BD8032194FB7C
:10064000F1F16429A8BF64210329ACBF5918D91C52
:1006500003F0BEF90368C3F30F13013B9C4208D2B9
:10066000A31C013464002A6840F8232044F00104EC
:100670004460002038BD01282DE9F84304DC1C202B
:10068000BDE8F84300F066BF02284E680CD08C68C5
:10069000E70709D56410012CB8BF0124F50705D57B
:1006A0004FF0FF30BDE8F8830124F7E7042EF7D9B7
:1006B00033680D6803F00F02042A23D1E80706D43B
:1006C000042D04D92B6803F00F03042B01D00E2056
:1006D000D6E73046FFF7EEFEA042E1DB304602F0FF
:1006E0009FFF0646284602F09BFF013C0146301959
:1006F00009F0BBFE0028D3D0801B0130400040F041
:100700000100CFE7092A38D177687F10BC42C7DCE7
:10071000E90729D4042D27D92B6803F00F03042BF4
:1007200022D1284602F07CFF804604F1010956F8E8
:100730002900854203D1640044F00100B2E7C207FA
:100740000ED404280CD9036803F00F03042B07D13F
:1007500002F066FF0146404609F04EFE0028EAD04E
:10076000B9454C46E1DD9BE7631C56F82320AA42BD
:10077000E1D0BB421C46F7DD92E7032A90D1C3F3D8
:100780000F17C3F34173C3EB8707BC4288DCEB0749
:1007900028D4042D26D9286800F00F03032B17D185
:1007A000C0F30F13C0F3417005F10408C0EB8300E0
:1007B0003F1A013C40440336BC423FF771AF321947
:1007C0004346834219460FD315D10134600096E7A2
:1007D000042B07D1284602F023FF80462846FFF766
:1007E00069FEE5E70F204BE712F8015F09788D42BB
:1007F00003F10103E5D00134DEE708B502F0F4FEB1
:10080000400040F0010008BDC30711D404280FD9EF
:10081000026802F00F03032B0AD101F00303C3F1B6
:1008200004035B0703F0C04322F0C042134303609C
:10083000704701282DE9F0470546884604DC1C2056
:10084000BDE8F04700F086BE4C6814F0010701D106
:100850000D20F5E7022802D08B68DA07F8D5D8F822
:100860000060F30700F1A980042E40F2A6803268F0
:100870006410012C02F00F03B8BF0124092B28D10A
:100880007668022D4FEA660605D0D8F808305B106E
:100890009E42A8BF1E46351B0135012225EAE5759B
:1008A000A918092003F058F8074648B16D0003461F
:1008B00045F00105D8F8002043F8045FA64202DAAB
:1008C0003846BDE8F087013452F8241043F8041F7D
:1008D000F4E7042B43D1304602F0A2FEFFF714FEEA
:1008E000022D824605D0D8F808305B109842A8BF88
:1008F0009A46A24504DA0020BDE8F04703F0A6B806
:10090000304602F08DFE0546A74222DB304602F05B
:1009100087FEA94606462846FFF7E2FD0134A245B8
:100920000546F8DAA0EB0905284603F08FF80746DC
:100930000028C5D002F074FE0446D8F8000002F08A
:100940006FFEA9EB060101442A46204609F09CF9F6
:10095000B6E72846FFF7C4FD01370546D4E7032B69
:100960002BD1C2F30F13022DC2F34172C2EB8302EB
:1009700005D0D8F808305B109A42A8BF1A46A242A8
:1009800006DA002211460320BDE8F04702F0E4BF7A
:10099000151B0423291D002291FBF3F1032002F013
:1009A000DBFF074600288BD001352946FFF72CFFD7
:1009B000E11C2A4631440430C8E7212040E70028E2
:1009C000F8B504DC1C20BDE8F84000F0C3BD0C689D
:1009D00014F001060FD0641024EAE474E11C002234
:1009E0008910032002F0B8FF054610B12146FFF739
:1009F0000BFF2846F8BD042C01D80025F9E725682F
:100A000005F00F05042D19D12046FFF753FD32469E
:100A1000C11C074691FBF5F1032002F09DFF05463E
:100A20000028E6D03946FFF7EFFE204602F0F8FD39
:100A30003A460146281D09F027F9DAE7092DDCD1ED
:100A400067687F100423F91C324691FBF3F1032001
:100A500002F082FF05460028CFD03946FFF7D4FECA
:100A60000434BE42C5DA54F8043FDA0742BFAA197B
:100A7000A3F3480313710136F3E77F2902DC017009
:100A800001307047B1F5006F0CDA03468A1162F04D
:100A90003F0203F8022B01F03F0161F07F0141703A
:100AA00018467047B1F5803F0FDA0B1363F01F0350
:100AB0000370C1F3851301F03F0163F07F0361F020
:100AC0007F014370817003307047B1F5883F0DDAC4
:100AD000F0230370902343708B1101F03F0163F00A
:100AE0007F0361F07F018370C170043070470000A4
:100AF0000028F7B50F4603DC1C2000F02BFD0CE0AE
:100B00000A6812F001000AD06C4651102046FFF727
:100B1000B4FF011B204602F0A0FF044616E0042AA1
:100B20003BD9136803F00F03092B36D155681C49D4
:100B30006D100124AC420CDD02F088FF044628B1A0
:100B40003F6802F06DFD0126AE421DDD204603B078
:100B5000F0BD013452F8243013F0010601D10D200C
:100B6000CBE75B107F2B09DDB3F5006F08DBB3F536
:100B7000803F07DB8B42D4BF042600263044D9E7F0
:100B80000226FBE70326F9E7013657F82610CB07C4
:100B9000E5D54910FFF771FFD6E72120ADE700BF8B
:100BA000FF0F010010B5044611F0010011D1042916
:100BB0000ED90B6803F00F03042B09D1084602F08D
:100BC0002FFD0146204609F017FCB0FA80F04009DD
:100BD00010BD0020FCE700000128F8B50E4604DC3B
:100BE0001C20BDE8F84000F0B5BC4D6815F00107C9
:100BF00006D1042D04D92B6803F00F02092A01D075
:100C00000B20EEE76C6809681F486410C3F30F13EC
:100C1000A34298BF03F1FF34FFF7C4FF40B10123A3
:100C2000BC4201DA0020F8BD013745F82730F7E76C
:100C300031681648FFF7B6FF50B1002CF2D0631CA4
:100C40000122013C944045F8232014436C60E9E7FD
:100C50003368DA0701D40D20C3E75B10002B0DDDEC
:100C60009C420BDB05EB830305EB84029A4207D120
:100C70000123013C9C4053601C43E7E71220B0E78E
:100C8000996843F8041FF1E777B300007BB30000D5
:100C9000002310B50B70C3070C4606D50E49421051
:100CA0002046BDE8104009F06BBB28B90B4920462F
:100CB000BDE8104009F084BB042801D10849F6E7DB
:100CC00009D9036803F00F03042B04D102F0A8FC38
:100CD00004490246E4E710BDB0BD000080B3000047
:100CE00086B300008BB300002DE9F04301288FB0DC
:100CF00081460E4607DC1C2000F02CFC05462846E9
:100D00000FB0BDE8F0830B6813F0010440F0A18040
:100D1000042B40F2D5801B6803F00F03092B40D150
:100D2000274656F8273013F0010806D1042B04D9C2
:100D3000186800F00F00092801D02220DCE75B686A
:100D40000137B94504EB6304EBD10122A11802F08D
:100D500003FE054608B90025D1E7640044F001040C
:100D60004460424600F1080456F822104B680868B7
:100D70005B10C0F30F10984298BF00F1FF330431AD
:100D80000020834207DC013223EAE373BA4204EB1A
:100D90008304E9DBB3E751F804CF44F820C0013005
:100DA000EFE7032B40F08C80274656F8270010F021
:100DB0000108C2D10428C0D9036803F00F02032A36
:100DC00038D1C3F30F12C3F34173C3EB82031C4446
:100DD0000137B945E9D10423E11C002291FBF3F16D
:100DE000032002F0B9FD05460028B4D02146FFF7E4
:100DF0000BFD00F1040956F82840E10720D4042C2B
:100E00001ED9206800F00F03032B19D1C0F30F1374
:100E1000C0F34170C0EB830003344B46A3EB0902DF
:100E2000824211DB08F101080028A8BF8144B845BF
:100E3000E1DB64E7042A80D1FFF73CFB0444C7E709
:100E40002046FFF737FBE7E714F8012F03F8012BE3
:100E5000E4E700252C4656F82500C20732D40428C2
:100E600030D9036803F00F02042A32D1FFF722FBC6
:100E700004440135A945EED1204602F0E7FD0546C0
:100E800000283FF468AF041DB04606EB890958F806
:100E9000046BF30728D4042E26D9336803F00F021D
:100EA000042A34D13046FFF705FB0746304602F0EE
:100EB000B7FB3A460146204608F0E6FE3C4421E0F6
:100EC0002546C8E701A9FFF7E3FE01A809F09EFA4D
:100ED000CEE7032A7FF431AFC3F30F12C3F341739C
:100EE000C3EB82031C44C4E701A93046FFF7D0FEE0
:100EF00001A809F08BFA01A906460246204608F02F
:100F0000C3FE3444C145C2D100232370F7E6032A4F
:100F1000F8D1C3F30F17C3F34173C3EB87073A4606
:100F2000311DC8E72DE9F04F002891B0894607DC54
:100F30001C2000F00FFB0446204611B0BDE8F08FE6
:100F40000C6814F0010706D1042C04D9236803F0BF
:100F50000F03092B01D00B20EBE766687610002EFB
:100F600003DC384602F072FDE5E701286BD04868E3
:100F7000C50768D4042866D9036803F00F03042B5F
:100F800061D102F04DFB0546284609F03FFA0434D2
:100F900006F1FF3A04EB860380460AFB00FB009350
:100FA00054F8040FC10750D404284ED9026802F047
:100FB0000F02042A50D1FFF77DFA009BA34283441D
:100FC000EED1584602F042FD04460028B4D0D9F8CC
:100FD00000B0B8F1000F04D0D9F8040002F020FBF3
:100FE0000546204602F01CFB0BF1040B81465BF822
:100FF000043F0093184602F013FB009BDA070146FA
:1010000001D4042B04D803A91846FFF741FE03A915
:101010000846019109F0FAF9019900900246484604
:1010200008F032FE009B9944B8F1000F07D0BA4592
:1010300005DD48464246294608F026FEC1440137F0
:10104000BE42D4D178E7064D9EE703A9FFF720FE04
:1010500003A809F0DBF9B0E702F0E2FAF9E700BF14
:101060001FB80000002810B511DD0B6813F0010453
:1010700002D05C1024EAE4740122A118092002F0D5
:101080006BFC18B1640044F00104446010BD0024FE
:10109000F2E70A6838B512F0010436D1042A34D9CF
:1010A0001368496803F00F00092818D15068C3F38A
:1010B0000F134010834298BF03F1FF30151DA0426B
:1010C00005DC01330220984205DB002038BD45F8DD
:1010D000041F0134F3E742F820100130F3E703283E
:1010E00013D1C80704D41320BDE8384000F032BA49
:1010F0004910FF29F7D80432C3F30F1302EB83031F
:101100009A42E2D202F8011BFAE70B2000F022FA21
:10111000DBE700002DE9F8434E6816F001080F46A2
:1011200027D1042E25D9346804F00F03092B10D1E0
:101130007568C4F30F146D10AC4200D8651E396891
:10114000CB071AD54C10002C01DDA54220DA122065
:1011500034E0042B04D13046FFF7ACF90546EEE746
:10116000032B08D1C4F30F15C4F34174C4EB8505F8
:10117000E5E70025E3E74546E1E72F48FFF712FDE5
:10118000B0B109F095F890FBF5F404FB15040134B7
:10119000B8F1000F4ED1042E4CD9336803F00F0381
:1011A000092B11D1013456F824402046BDE8F883BC
:1011B00039682248FFF7F6FC20B91120BDE8F84352
:1011C00000F0C8B92C46E3E7042B2BD1304602F0DF
:1011D00027FA0546FFF798F9A042B8DB012C1BDC83
:1011E000304602F01DFA81462846FFF779F9461B82
:1011F000304602F02BFC04460028D6D002F010FA4C
:101200008046786802F00CFAA5EB090101443246E9
:10121000404608F039FDC8E72846FFF761F9013C70
:101220000546DBE7032B05D13444E478640044F041
:101230000104BAE70B20C1E770B300007BB30000E4
:101240002DE9F0414C6814F0010688462ED1042C9B
:101250002CD923688F6803F00F02092A13D165681F
:10126000C3F30F136D10AB4200D85D1ED8F8001009
:101270002848FFF797FC68B3236803F00F03092B96
:101280001ED1012317E0032A10D1FA0704D413203A
:10129000BDE8F04100F05EB97E10FF2EF7D8C3F331
:1012A0000F15C3F34173C3EB8505DFE70B20EFE7B1
:1012B000013344F823709D42FADA0020BDE8F08142
:1012C000032BFAD1033401239D42F6DB04F8016FAE
:1012D0000133F9E7D8F80010CB0706D549100029EB
:1012E00001DD8D4208DA1220D2E70B48FFF75AFCE5
:1012F00008B91120CCE72946236803F00F03092B16
:1013000003D1013144F82170D7E7032B04BF6418DF
:10131000E670D2E777B300007BB30000086808B539
:10132000C3071BD4042819D9036803F00F02092A44
:1013300001D1406808BD032A09D1C3F30F12C3F3DA
:101340004170C0EB8200400040F00100F2E7042A47
:1013500004D102F065F9FFF7D7F8F4E70B20BDE8F8
:10136000084000F0F7B80000024A03480B2103F0E0
:10137000C5BF00BF18B3000010B3000000207047C5
:101380000420704701207047002002F05FBB00205E
:1013900070470020704700207047002070470020F1
:1013A0007047002070470020704700207047000001
:1013B000024A03480C2103F0A1BF00BF00B40000A3
:1013C00060B400007047000010B510F0010402D0B6
:1013D0004410204610BD042812D9026802F00F0202
:1013E000042A07D102F01CF90A222146BDE8104068
:1013F00009F0D0B8032A03D10A2221460430F5E7C8
:10140000014B0D221A70E4E77402002010F0010273
:1014100010B516D1042802D90268C2F30F1211F0D8
:10142000010310D1042902D90B68C3F30F139342AF
:1014300016D1043000EB83020331904205D3012022
:101440000BE00022EBE70023F1E710F8014B11F865
:10145000013F1CB9B3FA83F0400910BD9C42ECD0A7
:101460000020FAE72DE9F74F804689469A46304F2B
:10147000304E6AB102233B70012333603368DFF8DA
:10148000D0B00024FC54444504DB03B0BDE8F08F29
:101490003260F3E759F824003168C30707EB010510
:1014A000C1F5487105D5244A4310284608F034FF99
:1014B00004E0C8B9214A284608F02EFF1C4808F06D
:1014C000A5FF3060BAF1000F0CD008F1FF33A34242
:1014D00008DDB0F5487F05D2431C20223A54002293
:1014E000FA5433600134CEE7042801D1144AE2E70C
:1014F0001BD9026802F00F03042B06D1019102F000
:101500008FF8104A01990346CFE7092B03D14368AE
:101510005A465B10C9E7032B08D1C2F30F13C2F37D
:101520004172C2EB8303084ABFE70123074ABCE7C5
:101530007502002098050020B0BD000080B30000B7
:1015400086B30000DBC30000DFB60000EAB600008F
:10155000D0B60000014B18700020704774020020C4
:1015600010B501F091FD084C231D01461F221846BD
:1015700008F066FF08F04AFF04308008000140F0E0
:1015800004002060204610BD500200202DE9F04FDD
:1015900085B000F1180104690291D0E90232824657
:1015A00001EB8404BD4F4169029800EB8109397851
:1015B00003EB820529BB53F82230B94A1E1203F00F
:1015C0007F03043552F82330904643F00103184757
:1015D0009AF8010004F0DAFA00238AF8003021E0DA
:1015E0003B7873B92B681E1203F07F03043558F85B
:1015F0002330EAE7029B221DD31AD82B26DD1A23BB
:101600003B70DAF808209AF8023039789AF801002D
:10161000AA1A921043EA022204F0BEFA00238AF8C2
:1016200000303B70DAF80830ED1A029BE41AA9EB9F
:101630000309AD10A4104FEAA903CAF80C50CAF868
:101640001040CAF8143005B0BDE8F08F3B78266032
:101650000BB11446D5E72B681E1203F07F03144626
:1016600058F823300435B0E7029B221DD31AD82B3B
:1016700002DD1A233B70C4E72968216039782B1DED
:1016800011B114461D46BCE76B681E1203F07F03C0
:10169000144658F82330083597E7029B221DD31AC9
:1016A000D82B02DD1A233B70ABE73B7805EB8606AF
:1016B00026600BB11446A4E72B681E1203F07F03CB
:1016C000144658F8233004357FE7029B221DD31AB5
:1016D000D82B02DD1A233B7093E7724B53F8263068
:1016E00023603B780BB114468BE72B681E1203F086
:1016F0007F03144658F82330043566E7694B54F8E5
:10170000042D43F826203B78002B7FF47AAF2B681A
:101710001E1203F07F03043558F8233055E7614B60
:10172000009353F82600FFF74FFE834654F8040D4C
:10173000FFF74AFE5844009B400040F0010043F888
:1017400026003B78002B7FF45CAF2B681E1203F061
:101750007F03043558F8233037E7029B221DD31A44
:10176000D82B02DD1A233B704BE7029B4B4534BF5D
:1017700059F80C3C012323603B780BB1144640E739
:101780002B681E1203F07F03144658F823300435EB
:101790001BE7029B221DD31AD82B02DD1A233B70B4
:1017A0002FE7029B4B450FD259F80C3C06F18046BF
:1017B0005B10C3EB8373033E334459F8233023603B
:1017C0003B782BB114461CE718233B700023F6E747
:1017D0002B681E1203F07F03144658F8233004359B
:1017E000F3E6029B4B4519D259F80C3C54F8042CF3
:1017F0005B1006F18046C3EB8373033E3344043C25
:1018000049F823203B78002B7FF4FBAE2B681E1297
:1018100003F07F03043558F82330D6E618233B70D5
:10182000F0E7029B4B452DD259F80C3C06F180465F
:101830005B10033EC3EB8373334459F82300FFF777
:10184000C3FD221F834654F8040C0092FFF7BCFD31
:1018500059F80C3C009A5B10C3EB837358441E4448
:10186000400040F0010049F8260014463B78002B68
:101870007FF4C7AE2B681E1203F07F03043558F8BF
:101880002330A2E618233B70F0E7029B221DD31AF7
:10189000D82B09DD1A233B70B3E600BF7402002089
:1018A000D0B40000C48B012059F8263023603B7867
:1018B0000BB11446A5E62B681E1203F07F031446F5
:1018C00058F82330043580E654F8043D49F82630B2
:1018D0003B78002B7FF495AE2B681E1203F07F033C
:1018E000043558F8233070E659F826004FEA600BAB
:1018F00054F8040DFFF768FD584440003B7840F071
:10190000010049F82600002B7FF47BAE2B681E12E5
:1019100003F07F03043558F8233056E6029BA4EB0E
:101920008604A3420BD83B78002B7FF46AAE2B6869
:101930001E1203F07F03043558F8233045E6C348F0
:1019400001F05EFE3B78002B7FF45BAE2B681E122D
:1019500003F07F03043558F8233036E6002E05EBFC
:101960008605FFF65FAE3B78002B7FF44AAE2B680E
:101970001E1203F07F03043558F8233025E654F88F
:10198000043D042B04D1002E05EB8605FFF64AAE7C
:101990003B78002B7FF435AE2B681E1203F07F03DB
:1019A000043558F8233010E654F8043D042B04D0D5
:1019B000002E05EB8605FFF635AE3B78002B7FF455
:1019C00020AE2B681E1203F07F03043558F8233035
:1019D000FBE554F8040CC3070BD540100138002870
:1019E0000ADB400040F0010005EB860544F8040CDA
:1019F00018E6FFF7E9FCF1E73B78043C002B7FF4A5
:101A000000AE2B681E1203F07F03043558F8233014
:101A1000DBE5029B04F10C02D31AD82B02DD1A235A
:101A20003B70EEE5730003F4FF7343F001032360A2
:101A3000DAF80830EB1A9D109AF8023043EA0523D1
:101A40005B0043F001036360029BA9EB03035B109F
:101A500043F00103A3603412E6B27D4B8AF80240E2
:101A600091463A7853F83630CAF808301AB103F183
:101A700008054C46C5E503F10C059B681E1203F0F2
:101A80007F034C4658F823309FE5029B54F8046CC2
:101A90004B452AD1F1071BD4042E12D9336803F029
:101AA0000F03042B0ED1304601F0BAFD08F0AEFC56
:101AB0000630643003F05EFC70B9043DDDF8089038
:101AC000B0E507D0002E14BF4FF400700720F0E7F8
:101AD0000A20EEE70720ECE731469AF8010004F00F
:101AE00072F800238AF80030E8E759F80C3C5849AE
:101AF0005A106FF0030353430C3B09EB030449F8FE
:101B0000036059F8083C5A108AF80220D2B2C3F395
:101B1000552351F83220CAF8082059F8041C4FEA1E
:101B20006109029901EB89093978043402EB8305D4
:101B300000297FF466AD52F823301E1203F07F03B4
:101B4000043558F8233040E554F8040CFFF73CFC0A
:101B50001E288346A4EB860425DC00280BDC3B789A
:101B6000002B7FF44EAD2B681E1203F07F0304356B
:101B700058F8233029E501F077FAABF1030B354E25
:101B8000834401F071FAA0EB0B00B042F9D83B7826
:101B9000002B7FF436AD2B681E1203F07F03043553
:101BA00058F8233011E501238AF8003001F05CFA7F
:101BB0000A385844CAF8040034E554F8040CFFF716
:101BC00003FCA4EB8604061E0BDC3B78002B7FF4A1
:101BD00018AD2B681E1203F07F03043558F823302C
:101BE000F3E41D4B9E4202DD1D233B7009E50123FA
:101BF0008AF8003001F038FA4FF47A7303FB0600DC
:101C00000A38D7E700233046A4EB8604134E1A4661
:101C10002146FFF727FC3168114801F01EFF114BE8
:101C2000316818600E4803F075FE31680C4803F007
:101C3000CFFF3B78002B7FF4E4AC2B681E1203F03F
:101C40007F03043558F82330BFE400BFFCB6000022
:101C5000CC8301203F420F0080EE36009805002023
:101C600075020020080000203B78A4EB8604002BBE
:101C70007FF4C7AC2B681E1203F07F03043558F8BD
:101C80002330A2E4504603F0D9FB3B78002B7FF4CD
:101C9000B8AC2B681E1203F07F03043558F82330CC
:101CA00093E454F8043CB3BB54F80C3CDA0726D553
:101CB0005B105A0042F0010244F8082C002B3BDD77
:101CC0005A0042F0010244F8042C54F8082CC3EBEB
:101CD000620354F80C2CD10720D501335B0043F08C
:101CE000010349F826303B78002B7FF48AAC2B683F
:101CF0001E1203F07F03043558F8233065E4042BEB
:101D000006D91A6802F00F02092A01D15B68CFE7F1
:101D100019233B7075E45B10013BCFE7042A08D917
:101D2000116801F00F01092903D1023352F8233061
:101D3000D7E719233B7064E40435D4E7029A04EB37
:101D400086039B1AD82B10DC0122002E06F1FF33EC
:101D50000EDC3B78002B7FF454AC2B681E1203F092
:101D60007F03043558F823302FE41A233B7048E4EE
:101D700022601E460434E8E7029A231D9B1AD82BE2
:101D800002DD1A233B703CE4029B4B452AD254F8F7
:101D9000040CFFF719FB002821DD59F80C3C5B10FF
:101DA00083421CDBC3EB8373184400F1804004388A
:101DB000A4EB860359F820201A606FF0030303FB9D
:101DC00006443B780434002B7FF41BAC2B681E12B6
:101DD00003F07F03043558F82330FFF7F6BB2023C8
:101DE0003B70EAE71823FBE7C04B1A68A4EB8603B5
:101DF0001A606FF0030303FB06443B780434002BA6
:101E00007FF4FFAB2B681E1203F07F03043558F8F4
:101E10002330FFF7DABB54F8043C042B3B780CBFAB
:101E200005EB8605043C002B7FF4EBAB2B681E1200
:101E300003F07F03043558F82330FFF7C6BB54F88E
:101E4000043C042B1CBF002344F8043C3B78A4F161
:101E500004021CBF05EB8605224613B11446FFF7AA
:101E6000D0BB2B681E1203F07F03144658F82330B2
:101E70000435FFF7AABB002EA4EB860115DC1C235A
:101E80003B7000226FF0030303FB06443B780A60BB
:101E90000434002B7FF4B5AB2B681E1203F07F03D4
:101EA000043558F82330FFF790BB0B684FF0000C57
:101EB0005B1051F82C0010F0010202D10D233B7091
:101EC000E0E7401083420CF1010CA8BF03466645D1
:101ED000EFDC5B0043F00102D4E7002EA4EB8601A7
:101EE00015DC1C233B7000226FF0030303FB064448
:101EF0003B780A600434002B7FF483AB2B681E12FE
:101F000003F07F03043558F82330FFF75EBB0B68FE
:101F10004FF0000C5B1051F82C0010F0010202D1C0
:101F20000D233B70E0E7401083420CF1010CB8BF79
:101F300003466645EFDC5B0043F00102D4E754F84A
:101F4000080CFFF741FA834654F8040CFFF73CFAFB
:101F5000A4EB86038345B4BF0420002018606FF013
:101F6000030303FB06443B780434002B7FF449ABA6
:101F70002B681E1203F07F03043558F82330FFF757
:101F800024BB54F8080CFFF71FFA834654F8040CDE
:101F9000FFF71AFAA4EB86038345D4BF0420002080
:101FA00018606FF0030303FB06443B780434002BF6
:101FB0007FF427AB2B681E1203F07F03043558F81B
:101FC0002330FFF702BB54E902014FEA860B81423E
:101FD000A4EB0B0B14D10423CBF800306FF00303F8
:101FE00003FB06443B780434002B7FF40AAB2B68D8
:101FF0001E1203F07F03043558F82330FFF7E5BACB
:10200000042801D80023E7E7C307FBD4036803F0E3
:102010000F03042BF6D1CB07F4D40429F2D90B68B3
:1020200003F00F03042BEDD1FFF7F0F900280CBFEC
:1020300000230423D0E754E902014FEA860B8142D2
:10204000A4EB0B0B14D10023CBF800306FF003038B
:1020500003FB06443B780434002B7FF4D2AA2B68A0
:102060001E1203F07F03043558F82330FFF7ADBA92
:10207000042801D80423E7E7C307FBD4036803F06F
:102080000F03042BF6D1CB07F4D40429F2D90B6843
:1020900003F00F03042BEDD1FFF7B8F900280CBFB4
:1020A00004230023D0E754F8080CFFF78DF983468A
:1020B00054F8040CFFF788F9A4EB86038345ACBF02
:1020C0000420002018606FF0030303FB06443B78F4
:1020D0000434002B7FF495AA2B681E1203F07F03B3
:1020E000043558F82330FFF770BA00BF080000200D
:1020F00054F8080CFFF768F9834654F8040CFFF70E
:1021000063F9A4EB86038345CCBF0420002018604C
:102110006FF0030303FB06443B780434002B7FF489
:1021200070AA2B681E1203F07F03043558F8233081
:10213000FFF74BBA54F8043C042BA4EB860314BFFE
:10214000042200221A606FF0030303FB06443B786D
:102150000434002B7FF455AA2B681E1203F07F0372
:10216000043558F82330FFF730BA54F8080CFFF75D
:102170002BF9834654F8040CFFF726F95844A4EBD6
:102180008603400040F0010018606FF0030303FB7A
:1021900006443B780434002B7FF433AA2B681E12CC
:1021A00003F07F03043558F82330FFF70EBA54F8D4
:1021B000080CFFF709F9834654F8040CFFF704F9FB
:1021C000ABEB0000A4EB8603400040F00100186078
:1021D0006FF0030303FB06443B780434002B7FF4C9
:1021E00010AA2B681E1203F07F03043558F8233021
:1021F000FFF7EBB954F8080CFFF7E6F8834654F8FC
:10220000040CFFF7E1F800FB0BF0A4EB86034000A1
:1022100040F0010018606FF0030303FB06443B78B5
:102220000434002B7FF4EDA92B681E1203F07F030A
:10223000043558F82330FFF7C8B954F8040CFFF7F9
:10224000C3F88346B8B91F233B70A4EB8603C3F8D9
:1022500000B06FF0030303FB06443B780434002B0B
:102260007FF4CFA92B681E1203F07F03043558F8C2
:102270002330FFF7AAB954F8080CFFF7A5F890FB34
:10228000FBFB4FEA4B0B4BF0010BDEE754F8040C61
:10229000FFF79AF88346B8B91F233B70A4EB860377
:1022A000C3F800B06FF0030303FB06443B7804342B
:1022B000002B7FF4A6A92B681E1203F07F030435C0
:1022C00058F82330FFF781B954F8080CFFF77CF871
:1022D00090FBFBF303FB1B0B4FEA4B0B4BF0010B8B
:1022E000DCE754F8040CFFF76FF80028B8BF404251
:1022F000A4EB8603400040F0010018606FF0030378
:1023000003FB06443B780434002B7FF47AA92B6846
:102310001E1203F07F03043558F82330FFF755B938
:10232000A4EB860B012EDBF8000028D1FFF74CF858
:10233000324603460393009207F0BAFF039B009ACC
:10234000012BB8BF012390FBF3F101FB13031344EE
:102350005B0043F00103CBF800306FF0030303FB95
:1023600006443B780434002B7FF44BA92B681E12E3
:1023700003F07F03043558F82330FFF726B9FFF741
:1023800023F80090DBF80400FFF71EF8009A0130F4
:10239000831ACFE7A4EB860B5946304601F0F2FCD6
:1023A0006FF0030303FB06443B78CBF800000434D2
:1023B000002B7FF426A92B681E1203F07F0304353F
:1023C00058F82330FFF701B954F8080CFEF7FCFF6A
:1023D000834654F8040CFEF7F7FF0BEA0000A4EB69
:1023E0008603400040F0010018606FF0030303FB18
:1023F00006443B780434002B7FF403A92B681E129B
:1024000003F07F03043558F82330FFF7DEB854F8A3
:10241000080CFEF7D9FF834654F8040CFEF7D4FFEE
:102420004BEA0000A4EB8603400040F00100186076
:102430006FF0030303FB06443B780434002B7FF466
:10244000E0A82B681E1203F07F03043558F82330F0
:10245000FFF7BBB854F8080CFEF7B6FF834654F8F4
:10246000040CFEF7B1FF8BEA0000A4EB86034000EA
:1024700040F0010018606FF0030303FB06443B7853
:102480000434002B7FF4BDA82B681E1203F07F03D9
:10249000043558F82330FFF798B854F8040CFEF7C9
:1024A00093FFC043A4EB8603400040F00100186096
:1024B0006FF0030303FB06443B780434002B7FF4E6
:1024C000A0A82B681E1203F07F03043558F82330B0
:1024D000FFF77BB854F8080CFEF776FF834654F8F4
:1024E000040CFEF771FF0BFA00F0A4EB860340002A
:1024F00040F0010018606FF0030303FB06443B78D3
:102500000434002B7FF47DA82B681E1203F07F0398
:10251000043558F82330FFF758B854F8080CFEF784
:1025200053FF834654F8040CFEF74EFF4BFA00F0BD
:10253000A4EB8603400040F0010018606FF0030335
:1025400003FB06443B780434002B7FF45AA82B6825
:102550001E1203F07F03043558F82330FFF735B817
:1025600054F80C0CFEF730FF834654F8080CFEF7C5
:102570002BFF8BFB002354F8040CCDE90023FEF75E
:1025800023FFDDE90023C0F1200CB0F1200103FAA4
:102590000CFC22FA00F040EA0C005CBF43FA01F1A7
:1025A00008436FF00303A4EB860E400003FB0644D0
:1025B0003B7840F00100CEF800000434002B7FF49B
:1025C00020A82B681E1203F07F03043558F823302F
:1025D000FEF7FBBFA4EB860B59463046FEF742FDE3
:1025E0006FF0030303FB06443B78CBF80000043490
:1025F000002B7FF406A82B681E1203F07F0304351E
:1026000058F82330FEF7E1BFA4EB8604214630469C
:10261000FEF73FFD3B78002B7EF4F3AF2B681E12D4
:1026200003F07F03043558F82330FEF7CEBFA4EB48
:10263000860B59463046FEF76DFD6FF0030303FB32
:1026400006443B78CBF800000434002B7EF4D9AF6D
:102650002B681E1203F07F03043558F82330FEF771
:10266000B4BFA4EB860421463046FEF7E9FD3B7873
:10267000002B7EF4C6AF2B681E1203F07F030435D7
:1026800058F82330FEF7A1BFA4EB860B594630461D
:10269000FEF744FE6FF0030303FB06443B78CBF8E0
:1026A00000000434002B7EF4ACAF2B681E1203F044
:1026B0007F03043558F82330FEF787BF54F8040C25
:1026C00000F0AEFF54F8083CDA072AD4042B0CD9EA
:1026D0001B6803F00F03013B082B10D8DFE803F061
:1026E000052127230F0F0F0F2500C74907F084FE90
:1026F000A4EB8603002814BF002204221A606FF0A6
:10270000030303FB06443B780434002B7EF479AFCB
:102710002B681E1203F07F03043558F82330FEF7B0
:1027200054BFBA49E2E7BA49E0E7BA49DEE7BA4935
:10273000DCE7029B04F1040BABEB0303D82B03DDB6
:102740001A233B70FEF75DBF00F096FC3B7840001B
:1027500040F00100206013B15C46FEF752BF2B68C9
:102760001E1203F07F035C4658F823300435FEF751
:102770002CBF029B04F1040BABEB0303D82B03DD4E
:102780001A233B70FEF73DBF00F06EFCA34B03EA3B
:1027900040003B7840F00100206013B15C46FEF73A
:1027A00030BF2B681E1203F07F035C4658F82330BD
:1027B0000435FEF70ABF029B04F1040BABEB0303E5
:1027C000D82B03DD1A233B70FEF71BBF00F054FC2F
:1027D000934B1B6898423DBFC3F5830303F6371341
:1027E000C018C01A40003B7840F00100206013B1CF
:1027F0005C46FEF706BF2B681E1203F07F035C46A3
:1028000058F823300435FEF7E0BE00F035FC844B69
:1028100018603B78A4EB8604002B7EF4F2AE2B68A4
:102820001E1203F07F03043558F82330FEF7CDBEA7
:102830003046A4EB860701237A4E1A463946FEF746
:1028400011FE3068643002F095FD10B9043DFEF7CA
:10285000E9BE9AF801203168734803F0C8F90123F2
:102860008AF8003000F000FC704A336812680633C2
:1028700002FB0300CAF804003C46FEF7D3BE304614
:10288000A4EB8607674E012300223946FEF7EAFDD6
:102890003068643002F06EFD0028D7D0624802F044
:1028A00025FFDCE7FEF75CFE6FF00303A4EB860B6D
:1028B00003FB06443B78CBF800000434002B7EF485
:1028C000A0AE2B681E1203F07F03043558F82330A6
:1028D000FEF77BBE3B78A4EB8604002B7EF491AE22
:1028E0002B681E1203F07F03043558F82330FEF7DF
:1028F0006CBEA4EB860B584600F0F1FB6FF00303AF
:1029000003FB06443B78CBF800000434002B7EF434
:1029100078AE2B681E1203F07F03043558F823307D
:10292000FEF753BEA4EB860B584600F0DAFB6FF0BF
:10293000030303FB06443B78CBF800000434002B70
:102940007EF45FAE2B681E1203F07F03043558F847
:102950002330FEF73ABEA4EB860B5946304600F012
:10296000C3FB6FF0030303FB06443B78CBF8000086
:102970000434002B7EF445AE2B681E1203F07F0357
:10298000043558F82330FEF720BEA4EB8604204619
:1029900000F0DCFB3B78002B7EF433AE2B681E127C
:1029A00003F07F03043558F82330FEF70EBEA4EB86
:1029B000860B5946304600F003FC6FF0030303FB1F
:1029C00006443B78CBF800000434002B7EF419AEAB
:1029D0002B681E1203F07F03043558F82330FEF7EE
:1029E000F4BDA4EB8604204600F09CFC3B78002B51
:1029F0007EF407AE2B681E1203F07F03043558F8EF
:102A00002330FEF7E2BD00BF0CB7000014B7000092
:102A10001BB7000022B7000027B70000FEFFFF7FB2
:102A2000A005002098050020750200200400002069
:102A30000121304600F044FC3B78002B7EF4E1ADF0
:102A40002B681E1203F07F03043558F82330FEF77D
:102A5000BCBD0021304600F033FC3B78002B7EF4F7
:102A6000D0AD2B681E1203F07F03043558F82330D5
:102A7000FEF7ABBDA4EB860B584600F0E3FB6FF00E
:102A8000030303FB06443B78CBF800000434002B1F
:102A90007EF4B7AD2B681E1203F07F03043558F89F
:102AA0002330FEF792BDA4EB860B584600F0DEFB08
:102AB0006FF0030303FB06443B78CBF800000434BB
:102AC000002B7EF49EAD2B681E1203F07F030435AD
:102AD00058F82330FEF779BDA4EB8604204600F0B9
:102AE00099FB3B78002B7EF48CAD2B681E1203F013
:102AF0007F03043558F82330FEF767BDA4EB860446
:102B0000204603F031FC3B78002B7EF47AAD2B6835
:102B10001E1203F07F03043558F82330FEF755BD2D
:102B2000A4EB860B584603F0B5FC6FF0030303FBE0
:102B300006443B78CBF800000434002B7EF461ADF2
:102B40002B681E1203F07F03043558F82330FEF77C
:102B50003CBDA4EB8604204603F07CFB3B78002BB5
:102B60007EF44FAD2B681E1203F07F03043558F836
:102B70002330FEF72ABDA4EB860B584603F082FBF8
:102B80006FF0030303FB06443B78CBF800000434EA
:102B9000002B7EF436AD2B681E1203F07F03043544
:102BA00058F82330FEF711BDA4EB860421463046C9
:102BB00001F07AFB3B78002B7EF423AD2B681E12CC
:102BC00003F07F03043558F82330FEF7FEBCA4EB76
:102BD00086042146304601F08DF93B78002B7EF4C7
:102BE00010AD2B681E1203F07F03043558F8233014
:102BF000FEF7EBBCA4EB86042146304601F08AFACE
:102C00003B78002B7EF4FDAC2B681E1203F07F0393
:102C1000043558F82330FEF7D8BCA4EB86042146CF
:102C2000304601F09DFA3B78002B7EF4EAAC2B682D
:102C30001E1203F07F03043558F82330FEF7C5BC9D
:102C4000A4EB860B5946304603F0FEFC6FF00303FD
:102C500003FB06443B78CBF800000434002B7EF4E1
:102C6000D0AC2B681E1203F07F03043558F82330D4
:102C7000FEF7ABBCA4EB860B5946304603F0ECFCE8
:102C80006FF0030303FB06443B78CBF800000434E9
:102C9000002B7EF4B6AC2B681E1203F07F030435C4
:102CA00058F82330FEF791BCA4EB860B594630460A
:102CB00003F0DAFC6FF0030303FB06443B78CBF828
:102CC00000000434002B7EF49CAC2B681E1203F031
:102CD0007F03043558F82330FEF777BCA4EB860B4E
:102CE0005946304603F006FA6FF0030303FB06442F
:102CF0003B78CBF800000434002B7EF482AC2B68C8
:102D00001E1203F07F03043558F82330FEF75DBC34
:102D1000A4EB86042146304601F016F93B78002BDF
:102D20007EF46FAC2B681E1203F07F03043558F855
:102D30002330FEF74ABCA4EB86042146304601F05E
:102D400037FA3B78002B7EF45CAC2B681E1203F044
:102D50007F03043558F82330FEF737BCA4EB860B0D
:102D60005946304601F09EF96FF0030303FB064419
:102D70003B78CBF800000434002B7EF442AC2B6887
:102D80001E1203F07F03043558F82330FEF71DBCF4
:102D9000A4EB86042146304601F048F93B78002B2D
:102DA0007EF42FAC2B681E1203F07F03043558F815
:102DB0002330FEF70ABC029BE31A9B10A4EB8604A7
:102DC000CAF810302146304602F0D0FC3B78002B88
:102DD0007EF417AC2B681E1203F07F03043558F8FD
:102DE0002330FEF7F2BB029BE31A9B10A4EB860B89
:102DF000CAF810305946304602F0B8FC6FF00303B1
:102E000003FB06443B78CBF800000434002B7EF42F
:102E1000F8AB2B681E1203F07F03043558F82330FB
:102E2000FEF7D3BB2DE9F84F224D0023002B03F111
:102E3000FF3706DA01F0DAFA02F0C2FD02F036FFDF
:102E400019270026DFF878803046D8F80020B242F3
:102E500015DD2B68184C01339342A8BF00232B606B
:102E6000D5F80090F02303FB09F304EB030AE35CBD
:102E7000A346EBB1022B04D15046FEF787FB3B463D
:102E8000D4E7012B0ED108B900F0EEF8F02303FBD4
:102E900009F39B440949DBF80420821A8A429CBF4B
:102EA0000222E254F02303FB09F3E35C022BE3D09C
:102EB0000136CAE7000000206C7A01203F420F0073
:102EC0009C0500200B4B012200211A61C3F8041558
:102ED000C3F808150421C3F810154FF44031C3F8A6
:102EE00004131A60044B4FF480611960034B1A708D
:102EF000704700BF00A0004000E100E0C7050020CF
:102F000004207047F8B5D1E9004514F001002DD038
:102F100015F001002AD064101C2C3CD81F4F6D10F6
:102F200041F288363B5DAE42A8BF2E46012B05D04C
:102F30000121204604F0C6FD01233B55184B1B78A8
:102F40000BB9FFF7BFFF002D4FF00003154A0EDC51
:102F5000154940F2DC50FF25D65CB44204BF21F88D
:102F60001300D5540133042BF6D10420F8BDD15CF5
:102F70008C4203D10C4A22F81360F6E70133042B8C
:102F8000F5D10023D15CFF2901D1D454F2E70133FC
:102F9000042BF7D1E9E70020E8E700BFA8050020EF
:102FA000C70500201C0000200E00002070B5D1E9EC
:102FB000004514F001001BD015F0010018D064107A
:102FC0001D2C28BF1B24164E335D012B05D001217B
:102FD000204604F077FD01233355124B6D10A5F107
:102FE00010029A42104B04D94FF0FF321A600420AD
:102FF00070BD0E4A1C600E4B93FBF5F313800D4A17
:10300000127812B9FFF75EFFF1E70B4A01219164D4
:10301000D2F848150B449BB2C2F84035E7E700BF31
:10302000A805002090860100180000200C00002058
:1030300020A10700C705002000A00040002802DCF6
:103040001C20FEF787BA0120704704207047002833
:1030500002DC1C20FEF77EBA0B68DB0701D40D20D2
:10306000F8E7002070470000024B01221A64D3F8F1
:10307000400570470080004008B5FFF7F5FF4FF4AA
:103080007A73B0FBF3F008BD0048704788B70000C2
:103090001D20704770B5054D2B5C8B4204460E46D3
:1030A00002D004F00FFD2E5570BD00BFA805002012
:1030B00070B50024084D2646635D012B08D1002120
:1030C000204604F029FD0021204604F0FBFC665553
:1030D00001341D2CF0D170BDA805002070470F20D1
:1030E00070473B2070470000F8B50B68DA070746C9
:1030F0000D4604D40D20FEF72DFA012007E05B10E9
:10310000062B05D103F0CCF8400040F00100F8BDDB
:10311000F3D80C4A0C4E52F82340335D2BB10021FA
:10312000204604F0CFFC00233355012F06DD6B68E9
:10313000042B03D10221204604F0C4FC204604F0F5
:10314000CBFBE1E76CB70000A805002070B5046870
:10315000E20702D54568EB0704D40D20BDE87040B6
:10316000FEF7F8B964101C2C23D8124E335D012BE6
:1031700018D00121204604F0A5FC01231B2C335557
:1031800010D10D4BDA6E0D4B202AB8BF4FF0A04383
:1031900002F01F0203EB8203D3F8002742F44072CF
:1031A000C3F80027A5F34A012046BDE8704004F0AB
:1031B00037BC70BDA8050020DCC60000000300502D
:1031C00070B50C68E30704D40D20FEF7C3F90120A5
:1031D00070BD64101C2C14D8012814DD4B68042B1E
:1031E00014BF002502250A4E335DAB4204D02946A8
:1031F000204604F067FC3555204604F0A9FC012860
:1032000003D00020E4E70025EDE70420E0E700BF5D
:10321000A805002013B50A4A044692E80300226874
:103220006B46042A83E8030019464FF0020003D1DD
:1032300000F070FF02B010BD00F092FFFAE700BF8F
:1032400034B7000010B5084C63792BB1002105207C
:1032500004F038FC00236371052004F079FC002899
:103260000CBF0420002010BDA805002010B5084C9C
:10327000E37A2BB100210B2004F024FC0023E3723D
:103280000B2004F065FC00280CBF0420002010BDBA
:10329000A805002007480849084A012343604B60FD
:1032A00053600023C0F80035C1F80035C2F800357E
:1032B000704700BF00C001400010024000200240E3
:1032C0001C2870B504460D4625D8134E335C012BDF
:1032D00004D0012104F0F6FB012333551C2C12D13C
:1032E000FFF7D8FF0D4B1A6F0D4B202AB8BF4FF0D8
:1032F000A04302F01F0203EB8203D3F8002742F43D
:103300004072C3F80027291C204618BF0121BDE8E0
:10331000704004F001BC70BDA8050020DCC60000B0
:10332000000300500368D90702D40D20FEF712B93C
:1033300041680A1F514251415810FFF7C1BF0000B8
:10334000F8B5314CD4F84031B3B10023D4F840552E
:10335000C4F840312D4B186800280DDB2C4A117839
:10336000B1FA81F14909117004F0D6FB294B1B8891
:103370002B449BB2C4F84035234AD2F84431002B89
:1033800037D00021244ED2F84445C2F84411337896
:10339000224D0C3433B12B68032B03D8204AD05C68
:1033A00004F0BAFB2B681E4F01335A4202F00302AD
:1033B00003F0030358BF53422B600022042B19462D
:1033C00018D00133F81810F8010CFF2801D10122A0
:1033D000F4E702B12960012104F09EFB0123337060
:1033E0002A68104B33F812302344074A9BB2C2F8C4
:1033F0004435F8BD4FF0FF332B600023337004F5E4
:103400008C435033F1E700BF00A0004018000020BB
:10341000C60500200C000020C5050020A4050020E2
:103420001C0000200E000020094B0A4940F2DC522B
:103430001A805A809A80DA80074A00231370074A5C
:10344000FF20087048708870C8701360704700BF14
:103450000E0000201C000020C5050020A40500204F
:10346000024B4FF0FF321A60704700BF1800002077
:10347000024A0348062101F041BF00BF3CB70000EB
:10348000E2BE000038B54FF4E1311D4804F002F807
:103490001C4B03210122C3F80815002404211A61E2
:1034A000C3F810151A60C3F804454FF08043022199
:1034B000C3F818150A209A6004F008FA124A234645
:1034C000FF21995401331D2BFBD1104B104D0122CC
:1034D0001A6000200F4A042301461468002CFCD017
:1034E0002C681160013B44EA0020F6D10A4B01220E
:1034F0001A6004F029F9BDE8384001F013B800BFA4
:10350000EC79012000800040A805002000D0004098
:1035100008D5004000D1004004D00040F8B5064670
:103520000948094F0C4603F0F5FF8442A8BF044642
:103530003546AB1B9C4205DD384603F0F1FF05F82C
:10354000010BF6E72046F8BDEC7901200146014861
:1035500003F0A5BFEC790120C3070CD4064B1B6810
:10356000834208D8054B1B68984204D850F8043CA5
:10357000002B18BF18467047D0050020CC0500204E
:103580000B4908B50122002341F823200133642BA5
:10359000FAD1084B1A60084B084A1846002106F079
:1035A00097FB074B40F8043F064B186008BD00BF6F
:1035B000C48B012008000020D405002070670100A2
:1035C000A09D0500C8050020034B044A1A60044B67
:1035D000044A1A60FFF7D4BFD0050020D4050020AC
:1035E000CC050020446D0120044B1B681868C0F313
:1035F0000F10023820EAE070704700BFC8050020B5
:1036000000B59BB00246054901A806F0B9FE01A825
:1036100002F089F802F04AFBFCE700BF0FB8000097
:10362000C30713D4042802D812D00B48704703688C
:1036300003F00F03042B01D104307047092B09D08C
:10364000064A0748032B18BF1046704705487047C5
:10365000054870470548704780B30000FAB700007E
:1036600003B80000E9B7000086B30000F3B700001C
:10367000064B074900201A6843F8040CC2F30F12E6
:10368000023203EB82038B42F5D37047D80500204A
:10369000446D01202F4B304A1868304B2DE9F04122
:1036A0001C682F4D136803F00F01072928D81368F1
:1036B000C3F30F13023302EB8302AA42F2D3294968
:1036C000002251F82200FFF747FF41F822000132A3
:1036D000642AF6D1244A1068FFF73EFF1060234A9F
:1036E000106810B1FFF738FF1060214B214C1E68A5
:1036F0000021F0274FF03C08B14214DBBDE8F08117
:10370000C3F30F1302EB83039A42D0D01968CE079C
:1037100007D4884205D28C4203D351F8041C01B16E
:103720001960043BF0E707FB01F31A191B5D0BB9A5
:103730000131E1E71269551E08FB012204EB820208
:103740001832002DF4DB52F8040DFFF705FF013DA0
:103750001060F6E7D0050020D8050020CC05002039
:10376000446D0120C48B012008000020446D01201D
:103770009C0500206C7A0120C307F0B540D4214B92
:103780001C68A0423CD3204B1D68A84238D850F892
:10379000043CABBB03680246C3F30F13012673B9A5
:1037A000904242F8046C2BD0116851F8043C51F857
:1037B0002370176041F82320013B0A46EFE752F8D7
:1037C0002310CF0702EB830C18D48C4216D88D42FD
:1037D00014D351F8047C8FB90F6807F00F0EBEF1B7
:1037E000070F08D9CCF8007042F8043C0B680A6057
:1037F000C3F30F13E1E741F8046CD0E7013BCEE7D8
:10380000F0BD00BFD0050020CC0500200D4930B52B
:103810000D4C0B461A6853F8045CC2F30F12901C4F
:1038200065B18B4214BF0A46002243F8042C01EB19
:10383000800103EB8003A342ECD330BD12011A6078
:10384000F7E700BFD8050020446D0120144B2DE997
:10385000F041144C1E464FF000083268C2F30F17B7
:1038600012070FD07D1C9E424FEA850505D01846F1
:103870002A46314606F013FA03465A1904352B44FA
:10388000C2F80080023706EB8706A642E5D3E41AA9
:10389000A410013C044A24011C601360BDE8F081BF
:1038A000D8050020446D0120C80500202DE9F04115
:1038B0009AB0FFF7D9FB214D0746002455F82400A4
:1038C0000134FFF759FF642CF8D11D4B1868FFF73E
:1038D00053FF1C4B186808B1FFF74EFF1A4DDFF875
:1038E00074800026D8F800309E4218DBFFF78EFF68
:1038F000FFF7D0FEFFF7AAFFFFF7B6FB134B144903
:103900001B681B68C3F30F13C21B023B01A806F020
:1039100037FD01A801F007FF1AB0BDE8F0812B7850
:1039200013B90136F035DDE72C69013C002CF8DBDA
:1039300005EB84039869FFF71FFFF6E7C48B0120AE
:1039400008000020446D01206C7A0120C805002089
:10395000C9B700009C0500202DE9F8431B4C2368E3
:103960001B684D1CC3F30F139D420646884617463D
:10397000A1460CDBFFF79AFF23681B68C3F30F1304
:103980009D4204DB0A20BDE8F843FDF7E3BD08F1E2
:103990000202D9F800009B1A1B0140F822300023D4
:1039A00040F8043C06F00F06034646EA0816940069
:1039B00043F8046B0119083CC9F800101C44A342E9
:1039C00001D3BDE8F88343F8047BF8E7C80500207D
:1039D000F8B510F0010704460E462CD1174B1B68B2
:1039E000834228D8164B1B68834224D9154D286082
:1039F0000068012200F00F00FFF7AEFF2C682F6077
:103A00000546C0B12146043051F8042BC2F30F1211
:103A1000B242A8BF3246920006F036F9FFF728FE00
:103A200044F8045CFFF736FE2268074B44F8047C38
:103A3000134023602C462046F8BD00BFD00500206F
:103A4000CC050020446D0120F0FF0F00011D002275
:103A5000042091FBF0F1FFF77FBF38B5054608461B
:103A60000C46FFF7F3FF50B1C21C2B46591B8C428A
:103A700006DC002CACBF0419041C0023237138BDE4
:103A800013F8011B02F8011FF0E7F0B502289BB004
:103A90000C4604DC1C20FDF75DFD1BB0F0BD086882
:103AA000C20706D4042804D9036803F00F03042BCB
:103AB00001D00E20EFE74B6813F00107F9D1042B7A
:103AC000F7D91B6803F00F03042BF2D18B68DB07D7
:103AD00001D40D20DFE7FFF7A3FD06466068FFF77E
:103AE0009FFDA5681AAC014604F8647D6D10304650
:103AF00002F07CFF29466423224602F0D9FF2046CB
:103B000006F084FC01462046FFF7A7FFC5E700004A
:103B100010B50446ADF5806D10B9FFF797FF0BE0C7
:103B200002F08BFE0138062827D8DFE800F00808ED
:103B300010172804230000200DF5806D10BD2046CD
:103B400002F0F5FE011B2046FFF787FFF4E7204651
:103B500002F0A1FE400040F00100EDE769464FF49D
:103B60008062204602F0B1FE684606F04FFC014636
:103B70006846E9E704210348E6E70020CDE7042092
:103B8000DAE700BF58B80000022838B50C4604DC5C
:103B90001C20BDE83840FDF7DDBC0868C10706D42D
:103BA000042804D9036803F00F03042B01D00E206E
:103BB000EFE76368DA07FAD4042BF8D91B6803F03F
:103BC0000F03042BF3D1A368DB0701D40D20E0E73A
:103BD000FFF726FD05466068FFF722FDA468014651
:103BE0006410284602F002FF214602F03EFFBDE8C5
:103BF0003840FFF78DBF012838B50C4604DC1C2087
:103C0000BDE83840FDF7A6BC0868C10706D4042803
:103C100004D9036803F00F03042B01D00E20EFE753
:103C20006368DA07FAD4042BF8D91B6803F00F0392
:103C3000042BF3D1FFF7F4FC05466068FFF7F0FCB6
:103C40000146284602F0D2FE02F04EFF400040F04E
:103C5000010038BD012870B505460C4604DC1C2067
:103C6000BDE87040FDF776BC0868C10706D404289B
:103C700004D9036803F00F03042B01D00E20EFE7F3
:103C80006368DA07FAD4042BF8D91B6803F00F0332
:103C9000042BF3D1FFF7C4FC06466068FFF7C0FCB5
:103CA000022D014615D0A468E30712D564103046F2
:103CB00002F09CFE054602F0C0FD012812D1002C46
:103CC00002DD0135012C07D12846BDE87040FFF721
:103CD0001FBF4FF0FF34EAE7284602F036FE013CF2
:103CE0000546EFE70228EFD1002CEDDD0135012C70
:103CF000EAD000221146284602F051FE02F025FECD
:103D0000013C0546F3E70000086810B510F0010417
:103D10001AD0441007EE904A9FED187AF8EEE77A31
:103D200067EE877A17EE900A05F010FC04F01AF897
:103D30000022134B05F062FC03F0C6FF05F00EFFF6
:103D4000400040F0010010BD042812D9036803F0C0
:103D50000F03042B07D1FFF763FC0A22214606F06C
:103D600019FC0446D6E7032B03D10A22214604306E
:103D7000F5E70D20FDF7EEFBCCE700BFD3023739A6
:103D80000000D040086808B5C30706D4042804D949
:103D9000036803F00F03042B04D00E20BDE8084095
:103DA000FDF7D8BBFFF73CFC0378232B08BF01309D
:103DB0001022002106F0EEFB00F10053B3F1804F1A
:103DC00001D31420EAE7400040F0010008BD0000E4
:103DD000024A0348062101F091BA00BF28B800004A
:103DE00020B80000002070471E20FDF7B3BB1E2046
:103DF000FDF7B0BB1E20FDF7ADBB1E20FDF7AABB33
:103E00001E20FDF7A7BB1E20FDF7A4BB1E20FDF75B
:103E1000A1BB1E20FDF79EBB1E20FDF79BBB1E20F5
:103E2000FDF798BB024A03480B2101F067BA00BFB7
:103E300094B80000ECB80000034B01221A60034B59
:103E40001868904010437047646D0120486D012050
:103E50002DE9F041EFF31082012302F0010883F312
:103E600010881549154C0968154D164E01398B40BF
:103E700003274FF00E0C4FF00B0E002B18D02168CB
:103E8000296018420AD0724611000139FDDC216810
:103E9000316039000139FDDC5B08EEE7390001399A
:103EA000FDDC21683160624611000139FDDCF3E779
:103EB00088F31088BDE8F08120000020586D0120B3
:103EC000080500500C05005070B5084E084D002440
:103ED00056F824000021FFF7DDF855F824000021F2
:103EE0000134FFF7D7F8052CF2D170BD84B900007A
:103EF000D0BC000008B5054B00221A60044B1B68BB
:103F00000BB102F039FC002008BD00BF606D01203C
:103F10005078012010B5041E0ADA0024074B53F82C
:103F2000242001239340064A1360064A136010BD03
:103F3000FFF7AEF8A042F0DDF0E700BFDCC60000FE
:103F4000586D0120180500502DE9F843344B1B68CB
:103F50000C461BB94FF0FF30FFF7DCFF246814F06C
:103F6000010525D0C4F34743C4F34720C4F34702F7
:103F700040F2596540435B4390FBF5F193FBF5F04C
:103F8000000240EA01401346534393FBF5F3184304
:103F9000244B1B68202B01BF234BC4F3456453F80B
:103FA000243043EA0020FFF753FF0020BDE8F883E8
:103FB000042CFAD9236803F00F03092BF5D154F828
:103FC000046FDFF86080DFF86090761040F2596788
:103FD000B542EADA54F8042FD3071FD5C2F347439A
:103FE000C2F34720C2F3470140435B4390FBF7FC19
:103FF00093FBF7F0000240EA0C400B464B4393FB67
:10400000F7F31843D8F80030202B02BFC2F3456203
:1040100059F8223043EA0020FFF71AFF0135D7E7AD
:10402000586D01202000002074BB000008B50B680B
:10403000DA074CBF5B104FF0FF3301280DDD4A68F3
:10404000042A14BF18222022054918460A60FFF7E7
:1040500045F8FFF75FFF002008BD1822F4E700BF16
:104060002000002010B510F0010402D044102046BA
:1040700010BD042812D9026802F00F02042A07D1E9
:10408000FFF7CEFA0A222146BDE8104006F082BAB8
:10409000032A03D10A2221460430F5E70D20FDF75B
:1040A00059FAE4E7086810F0010370B51CD0FFF777
:1040B000D9FF0346203B5E2B27D8154C03EB830327
:1040C0000022012110462344052A1AD09E5C0524B3
:1040D00010252E4218BF4018013C4FEA41014FEA1B
:1040E0006505F6D10132EFE70428E3D9026802F052
:1040F0000F010429DED1C2F30F13002BDAD00379AC
:10410000D8E7400040F0010070BD0120FCE700BF8F
:1041100098B9000038B508680D46FFF7A3FF0446BC
:104120006868FFF79FFF621E042A014612D8431EEB
:10413000042B0FD8084803EB8303134405680122BE
:1041400002FA03F32B430360044B1B6813B12046B0
:1041500002F013FB002038BD606D01205078012073
:1041600038B508680D46FFF77DFF04466868FFF71D
:1041700079FF621E042A014614D8431E042B11D86D
:10418000094803EB83031344012202FA03F3026894
:1041900022EA0302054B02601B681BB10022204685
:1041A00002F0EBFA002038BD606D0120507801204C
:1041B0002DE9F04F054685B008680C46FFF752FF21
:1041C000022D01903CDD6068FFF74CFF0746A068B8
:1041D000FFF748FF0446231DDFF8C8A00293661EC0
:1041E0004FF00108029B9E4206F1010935D006EB13
:1041F0008602531E07F1050B3D460393AB4522D0C3
:10420000042E19D86A1E042A16D8039B019ADAF8DC
:1042100000005919224B4FF0010C18EA020E0CFA5B
:1042200001F11B6811D00143CAF8001023B16246A6
:104230004946284602F0A1FA4FEA48080135DDE771
:1042400001242746C7E74E46CCE720EA0101CAF819
:104250000010002BF0D07246EAE73D1D042D1BD85C
:10426000012C19D1DFF83C80DFF834900026D8F813
:10427000003004FA05F223EA0203C8F80030D9F846
:104280000030013623B100223146781D02F075FA64
:10429000052E05F10505EAD1002005B0BDE8F08F37
:1042A00050780120606D0120086808B5C30703D568
:1042B000FFF7D8FE054B1860054B1B681BB1034B7D
:1042C000186802F05BFA002008BD00BF606D012095
:1042D000507801202DE9F3413F4D4FF441732C6894
:1042E000ADF804300A238DF806305CBBFFF7ECFD17
:1042F000DFF8F480264658F8267001213846FEF78C
:10430000C9FE01360021384603F006FC052EF2D125
:1043100000260DF1040816F8087001213846FEF752
:10432000B9FE01360121384603F0F6FB032EF2D127
:10433000FEF79AFE294B186001232B60204602B03D
:10434000BDE8F081012C1CD1244C2668FEF78CFEC0
:10435000864298BF801BC72801D80024EEE70021C1
:104360000420FEF797FE00210320FEF793FE0021B4
:104370000A20FEF78FFEFEF777FE022320602B60F7
:10438000EBE7022C21D1154B1C68FEF76DFE844231
:1043900098BF001BB0F57A6FDFD3042003F09CFABE
:1043A0000446032003F098FA06460A2003F094FA24
:1043B00034442044C0F53F6003230D3090FBF3F0FC
:1043C000074B1860012003F087FA064A00232B6090
:1043D00013600124B2E700BF546D01205C6D012021
:1043E000486D0120646D0120D0BC00002DE9F84328
:1043F000434E326852B9434B1B683BB9424B1B6872
:10440000002B74D0BDE8F843FFF764BF3F4D2C6824
:1044100084BB3D4B1B68002B65D13A4A336810685A
:104420001146002865D13A4F3A4EDFF8F4800B6010
:10443000002157F82400FEF72DFE56F824900121A4
:104440004846FEF727FEB9F1220F10D858F8292068
:10445000314B1F2AD8BF4FF0A04302F01F0203EBDD
:104460008203D3F8002742F44072C3F800270134D6
:10447000052CDDD12B68264EDFF88890254F002BC8
:10448000CCBF03F1FF330423002156F82300FEF7CD
:1044900001FE2A68214B53F82280002404EB84019A
:1044A00001EB0803D9F8001057F82400194101F076
:1044B0000101013403F030FB052CEFD12B68012101
:1044C00056F82300FEF7E6FD2B68002156F823007E
:1044D00003F022FB2B68013393FBF4F404EB840418
:1044E0001C1B2C6003E0FFF7F5FE002895D1BDE80A
:1044F000F883002B97D11360BDE8F843FFF7E4BCC5
:10450000606D0120506D0120646D01204C6D012013
:1045100084B90000D0BC00000003005074BC00004F
:10452000DCC600004FF0FF30FFF7F4BC024A03483E
:10453000092100F0E3BE00BF88BC0000E4BC00001D
:104540004FF0805310B51A69094B0224C3F8044593
:1045500022F00302884203D30022C3F8042510BDD1
:10456000D3F80044002CFBD0C3F808051044F1E751
:1045700000E00140002815BF4FF4D2214FF4B421D0
:104580004FF4B4204FF49620FFF7DABF00280CBF99
:104590004FF496234FF4B4231868030E532B0CBF2B
:1045A00020F07F4000207047064B0122C3F804250D
:1045B000D3F80024002AFBD000220160C3F80425B0
:1045C000704700BF00E00140002821F07F4141F02A
:1045D000A6410CBF4FF496204FF4B420FFF7E4BF80
:1045E0000A4B30B50124C3F80445002903DC00223E
:1045F000C3F8042530BD52F8044BD3F80054002D05
:10460000FBD040F8044B0139EFE700BF00E0014068
:1046100038B54C68023405460A462146FFF7E0FFEC
:1046200005EB840038BD0000124B1B68002B0BBF4C
:104630004FF4B4224FF4D2224FF496234FF4B42314
:1046400028B91A1DDB79522B08BF104670478242E9
:104650000DD9C378522B0AD14368023300EB830093
:10466000824204D9C378522B18BF00207047002023
:10467000704700BF686E01202DE9F0410020B4B002
:10468000FFF7D2FF0024DFF8A48005462746264620
:104690004DBB224D2868FFF779FF3B463246CDE9F6
:1046A00000401F4902A805F06BFE02A801F03BF88C
:1046B0001C4B1A682B68002B0CBF4FF496234FF449
:1046C000B423D21A4FF4704164235343009193FBF7
:1046D000F1F302A8144905F053FE02A801F023F8F3
:1046E00034B0BDE8F08169682A6801918B1C1F44D1
:1046F000D1B2C2F307239C42C2F30742009102A841
:104700004146B8BF1C4605F03BFE02A801F00BF87D
:104710002846FFF789FF01360546B9E7686E012094
:10472000EEBD00006C6E012098BD0000DABD0000F7
:1047300070B50020FFF72AFF05460120FFF726FF8E
:104740000C4B1E68B6FA86F485424FEA5414B8BF83
:10475000054620461C60FFF70DFF074A074B002E59
:1047600018BF1346064A691C2046BDE87040136016
:10477000FFF72ABF686E012004B0040004A0050002
:104780006C6E012070B50020FFF700FF024601208B
:10479000FFF7FCFE1F4E204C054672B968B94FF476
:1047A000D2214FF49620FFF7CBFE01212846FFF7D8
:1047B0000BFF1A4B3560236029E0AA4208DD002375
:1047C0003360164B23604FF4B4212368002017E0B8
:1047D00001233360124B23604FF4D221F5E7120E10
:1047E000522A08D000B123600E4800F09CFFBDE8BB
:1047F0007040FFF79DBF5A68023203EB820301202D
:104800008B4205D21A68551CE9D10028D3D170BD5E
:104810002160FCE7686E01206C6E012004B004008A
:1048200004A00500B3BD000010B50020FFF7FCFE9A
:10483000014608B9084610BD8478FFF7F5FEDA2C6A
:1048400008BF0146F5E700002DE9F04F4FF48072F4
:104850009FB0604C6048DFF880B1002105F038FA65
:104860004FF4807200215D4805F032FAD4F80090D0
:10487000B9FA89F84FEA58184046FFF77BFE0294D0
:10488000574A584C0020B9F1000F08BF1446FFF7F3
:10489000CBFF064626BB4846FFF778FE411C404644
:1048A000FFF792FE029BB9F1000FC3F800804E4B58
:1048B00014BF4FF496224FF4B4221C60A21A4FF496
:1048C000704164235343009193FBF1F305A84749DA
:1048D00005F056FD05A800F026FF1FB0BDE8F08FDB
:1048E0003568C5F30743A3F10A02092AC5F3072572
:1048F00047D81BF8051091BB10223D48DFF8F0A007
:1049000005F0E6F937463A68C2F307218D4209D12E
:10491000C2F307410B2927D013292CD00A2901D132
:10492000CAF800703846FFF77FFE07460028EAD134
:104930002F4F396881B12046FFF76AFE01230446F4
:1049400057F8231029B120460393FFF761FE039B1C
:1049500004460133042BF3D101230BF80530304614
:10496000FFF762FE064695E7D2B2022ADADC0AEBCE
:1049700082025760D6E710220021504605F0A8F9C0
:10498000D0E7A3F11502082AE9D8144A525D002A9B
:10499000E5D1152B0CBF3146002130460368C3F327
:1049A0000742152A0FD01D2A08BF0021FFF73CFE41
:1049B0000028F3D119B12046FFF72AFE0446074A22
:1049C00001235355CBE7C3F307239D4208BF01469C
:1049D000ECE700BF686E0120686D0120706E012059
:1049E00004A0050004B004006C6E01207DBD000031
:1049F000548D0120FFF728BF2DE9F84FDFF8A8B04C
:104A0000274F03339246042293FBF2F6DBF8003083
:104A1000B41C002B3B684FEA84040CBF4FF4B42253
:104A20004FF4D22223449A4281460D46B84614D20E
:104A3000FFF70AFFDBF80030002B3B680CBF4FF498
:104A4000B4224FF4D22223449A4206D2154800F0F1
:104A50006AFE00273846BDE8F88F2D025FFA8AF11A
:104A600041F0A441ADB2D8F800700D434FEA0941BE
:104A700001F47F0129433846FFF796FD07F1080549
:104A80003146381DC8F80050FFF78EFD1EB10A9A56
:104A90002846FFF7A5FD083C2544C8F80050D9E793
:104AA0006C6E012057BD0000686E012030B59BB0D0
:104AB000FFF768FE00214FF4FF621D4805F008F97A
:104AC000FFF7B2FE1A490024A0B9194B024653F869
:104AD000301001B101320130FF28F8D1154901A889
:104AE00005F04EFC01A800F01EFE134800F01BFE6E
:104AF0001BB030BD0368C3F307420A2A0BD1C3F3CE
:104B00000722FF2A04D001EBC20541F832002B71C5
:104B1000FFF78AFDD8E7132AFAD1C3F30723FF2B47
:104B20001EBF01EBC30241F833401471F0E700BF30
:104B3000CC83012023BE000037BE00000A4B0022B8
:104B4000C3F8002101225A60D3F80021002AFBD0CB
:104B50000022C3F80C2101229A60044B0222C3F800
:104B600080211A60704700BF0010004000E100E0A3
:104B7000074B0222C3F88020064B0022C3F8102105
:104B800001221A61D3F81021002AFBD0704700BF20
:104B900000E100E00010004008B504490A780AB1BD
:104BA000FFF7E6FF0020087008BD00BF716F01200D
:104BB0004FF08053586E400040F0010070470000F5
:104BC000024B1868400040F001007047F46F01206C
:104BD000024B1868400040F001007047240000209C
:104BE000024B1868400040F001007047F86F012048
:104BF00070B504460D461646FEF73EFA4FF0805358
:104C000001225B6E6270E270020A23F00043A2711F
:104C1000020CE2711A0A002160716372000EA27226
:104C20001A0C1B0E2670A17025712072E27223737C
:104C300070BD000010B5054C204605F0E7FB0146AD
:104C40002046BDE81040FEF708BF00BFFD6F012001
:104C5000104B1B685A1C10B514D0CBB1012B13D0CC
:104C6000022B13D0042B13D00B4C0C4A052B08BF7E
:104C70001446204605F0CAFB01462046BDE8104018
:104C8000FEF7EBBE064CF4E7044CF2E7054CF0E708
:104C9000054CEEE728000020CDBE0000D3BE00008A
:104CA000C8BE00001BB7000014B7000010B52148B3
:104CB0000278002A3DD14FF08043C3F80021012241
:104CC0001A60D3F80021002AFBD01B4B1B4C00229A
:104CD0000721C3F80C25C3F808151949C3F8102596
:104CE000C3F81C15C3F824250121C3F82C2508227C
:104CF000C3F83015C3F81425C3F818450224C3F8C7
:104D000034454FF6FF74C3F83C450E4CC3F83845A4
:104D10001824C3F85445C3F80423D3F8002242F002
:104D20001002C3F80022084AC3F80425FFF706FF63
:104D3000017010BD716F01200010004020000402BE
:104D40007469627521100100726F0120F8B5104B73
:104D50001B7804460BB9FFF7A9FF0E4E3378ABB1B1
:104D60000D4A1278D21A02F003010C4A02EB4112EA
:104D700002F1200710685168254603C50832BA427F
:104D80002C46F7D1013B33700120F8BD1846FCE7F3
:104D9000716F0120FC6F0120706F0120726F012084
:104DA00030B5002889B02ADD0D6815F0010426D140
:104DB000042D26D92B6803F00F03092B21D16B6832
:104DC0003F2B1EDD6846FFF7C1FFB0B19DF8002004
:104DD0000435A242A8BF1DF8043004F10104A6BFA7
:104DE0005B0043F001030123202C45F8043FF0D180
:104DF000054BDDF809201A60042009B030BD002001
:104E0000FBE72046F9E700BFF86F012030B5384BCB
:104E10001B788BB00BB9FFF749FF02A8FFF796FF8D
:104E200010B900200BB030BD9DF808300B2BF8D91D
:104E30009DF80930012BF4D19DF80B30012BF0D1F6
:104E40002C4D2D4C2D4ADDF8111000232B602370C2
:104E50009DF80C3013602A4A116023B9DDF8153033
:104E60002B6000230FE0012B11D1DDF815309DF8E8
:104E700019202B600DF11A010E239342A8BF13468F
:104E800000229A4230D10022E2540420CAE7022BC9
:104E900005D19DF8152012230DF11601EDE7042B25
:104EA0000DD10AAA6B4652F8130D516803C3DDE910
:104EB000000102F07DFE04F051FE2860D1E7052BD1
:104EC000CFD10AAA6B4652F8130D516803C3DDE92E
:104ED000000102F06DFE04F041FE9DF81D202860E7
:104EE0000A230DF11E01C8E7885CA0540132C8E70F
:104EF000716F0120F46F0120FD6F01202800002058
:104F0000F86F012010B5154B1B7804460BB9FFF75D
:104F1000CDFEFFF72DFE124B0022C3F80445C3F867
:104F2000002101221A60D3F80021002AFBD00022C0
:104F3000C3F80C2101229A60094AD2F80C31002BE7
:104F4000FBD0084B1978084B03EB4113C2F804352A
:104F5000FFF70EFEBDE81040FFF7F0BD716F0120B6
:104F600000100040706F0120726F012000B5002812
:104F700089B01DDD0B6813F0010219D1042B17D97C
:104F8000196801F00F01092912D159683F290FDD75
:104F9000043353F8040F10F0010118BFC0F34701A8
:104FA0000DF802100132202AF3D16846FFF7AAFF5C
:104FB000002009B05DF804FB002810B511DD0C6875
:104FC000E3070ED56410532C0BD8074B1B780BB995
:104FD000FFF76CFEFFF7CCFD044BC3F80845FFF765
:104FE000ADFD002010BD00BF716F0120001000401A
:104FF000002810B50DDD0C68E3070AD56410FF2CFE
:1050000007D8054B1B780BB9FFF750FE034BC3F8CD
:105010002445002010BD00BF716F0120001000402A
:10502000002813B515DD0C68E10712D564100A4A93
:105030000A4B072CCDE900230BD8094B1B780BB981
:10504000FFF734FE02AB1C44064B14F9082CC3F8DE
:105050000C25002002B010BDE2ECF0F4F8FC0004D6
:10506000716F01200010004070B5002888B020DD6D
:10507000086810F001041CD104281AD9036803F051
:105080000F03042B15D1FEF7CBFA064605F0BEF947
:10509000122828BF1220054600F10D0202216846A1
:1050A000FFF7A6FD8DF80D50A54205DC6846FFF719
:1050B00029FF002008B070BD0DEB0403325D9A7328
:1050C0000134F1E72DE9F041012888B00D4630DDCB
:1050D000086810F001042CD104282AD9036803F0D1
:1050E0000F03042B25D14B68DB0722D5FEF798FA76
:1050F000804605F08BF96D680E2828BF0E206E10D3
:10510000074600F1110201216846FFF771FD6B129D
:105110008DF80D606D14360E8DF80E308DF80F5031
:105120008DF810608DF81170A74206DC6846FFF715
:10513000E9FE002008B0BDE8F0810DEB040318F88B
:1051400004209A740134EFE730B5002889B016DDE9
:105150000C68E30713D56510684610220021FFF79D
:1051600047FD63128DF80D5064142D0E68468DF8BE
:105170000E308DF80F408DF81050FFF7C3FE002061
:1051800009B030BD174BD3F8002122B10022C3F87B
:10519000002101229A60D3F80C2102B30021C3F848
:1051A0000C11D3F80024012A0F4A19D1D3F848353D
:1051B0005B4213600D4A1378032B9CBF01331370BD
:1051C0000B4A1378013303F003031370094A02EB0F
:1051D0004313044AC2F80435024B01229A60704717
:1051E0001160F9E70010004024000020FC6F01204E
:1051F000706F0120726F0120024A0348102100F0F5
:105200007DB800BF48BE00003FBE0000044A05490B
:105210001368C8540133C3F309031360704700BF18
:105220002C7401202C70012070B51149114A0B68B3
:10523000834202DC00230B6017E0855CA5F1FA06CF
:10524000012E00F1010405D89C420FDAA55C013D56
:105250001F2D01D92046EBE70446151A165D2E5581
:105260000134A342FADC181A086070BD1570FAE721
:10527000387801203874012008B5FDF7F5FE074B9A
:105280001A68824284BF00221A601B68C01A44F662
:105290002063984294BF0020012008BD287001209F
:1052A00070B5094C094D0A4E23682A68934200D113
:1052B00070BDF05CFEF74AF90028F9D0236801338D
:1052C000C3F309032360EFE7307401202C7401203D
:1052D0002C70012070B5074E074D044633682A68CC
:1052E0009B1ADB43C3F30903A34200DB70BDFFF746
:1052F000D7FFF3E72C74012030740120F0B5074D7F
:105300002B680B2B08DC064F0C245C433E19C6E9C6
:105310000112013338512B60F0BD00BF34740120FD
:10532000648D012008B5FCF71FF8FFF7FFF8FCF7C4
:105330003FF8FEF79DF8FEF74BFDFEF773FDFFF714
:105340005BFF01F007F801F01BFABDE8084001F02F
:105350004FBC000008B54FF416620021034804F06A
:10536000B7FC034B00221A6008BD00BF6C7A012015
:105370009C050020064B074A1B6812689B1ADB43FA
:10538000C3F309038342D4BF00200120704700BF4C
:105390002C74012030740120F8B507460E461446DF
:1053A0001D4673B90320FFF7E5FF10B3FA20FFF79E
:1053B0002DFFF8B2FFF72AFFF0B2BDE8F840FFF783
:1053C00025BF501DFFF7D6FF98B1FB20FFF71EFF4A
:1053D000F8B2FFF71BFFF0B2FFF718FFE0B2FFF7DC
:1053E00015FFC4F30720FFF711FF2E46731B9C42E5
:1053F00000DCF8BD16F8010BFFF708FFF6E7000028
:10540000F8B50C4E0C4D0024F0273368A34203DCA2
:10541000BDE8F840FFF79EBF07FB04F359195B5D39
:105420002BB100231A4649781120FFF7B5FF01344C
:10543000EBE700BF9C0500206C7A0120F8B50E4C0C
:105440000E4E07460025BC4205F1010511D0237818
:1054500053B100231A4661781120FFF79DFFF02217
:105460000021204604F034FC0A2D04F1F004EAD1B6
:10547000F8BD3560F8E700BF6C7A01209C0500207C
:105480002DE9F04F12F00106ADF54F7D82468B46B7
:1054900017D001238DF8143042FA03F354128DF81B
:1054A000153052141B0E8DF817208DF818308DF81A
:1054B000164005AB0522FFF76FFF0DF54F7DBDE8E8
:1054C000F08F042A1FD9116801F00F03042B2BD190
:1054D00005AD022310462B70FEF7A2F8044604F037
:1054E00095FF40F22332904228BF1046621EB04220
:1054F00004DC2B46421C59465046DCE7013612F8C4
:10550000013FAB55F3E740F0C880A2F1040CDCF199
:1055100000024FF0030342EB0C028DF814308DF8BB
:10552000152005AB0222E6E7092B40F091801546D5
:1055300004238DF8143055F8043F4FEA6308B8F19E
:10554000200F8DF815804FEA6323A8BF4FF0200885
:105550008DF816308DF8178006AC03220521B04572
:1055600002DC05ABE21AC6E755F8040F10F001079C
:1055700006D1042847D9036803F00F03022B0DD18D
:105580004FF0010323704310637047121B0E401449
:10559000A770E070237105340136E0E7042B30D1A9
:1055A00023464FF0020C03F802CBCDE90121009312
:1055B0000393FEF735F8814604F028FF0C28DDE957
:1055C00001210AD8009B6070874201D1DC19E3E712
:1055D00019F80740DC550137F6E723460C2003F89D
:1055E000010F09F1FF3009F1080910F8017F03F8F4
:1055F000017F4845F9D12E23E372237363730E3480
:10560000CAE7012B08D12346071F03F8022B784273
:10561000784160701C46BFE7092B09D10423237031
:105620004368581060705B12A370E7700434B3E7EE
:10563000032B0AD121700368C3F30F10C3F3417326
:10564000C3EB800363701B12EEE727700134A3E7FE
:10565000032B7FF432AF05238DF81430C1F30F1301
:10566000C1F34171C1EB83010B1264298DF816302F
:105670000B46A8BF64238DF817308DF81510033240
:10568000DBB29E4202DB05AB0A1D34E705A83044BD
:1056900012F8014F04710136F3E7002A7FF40DAFD1
:1056A00033E700000F4970B5F022002402FB041319
:1056B0005D78854203D001340A2CF7D170BDF02209
:1056C0001846002104F004FB074A1368013BA3427B
:1056D00000D11460002329461A461120BDE870400D
:1056E000FFF75ABE6C7A01209C05002030B5B3B09C
:1056F00032AC0223054604F8C83D04F087FEC728F3
:1057000028BFC720691E0023984207DC421C23469D
:10571000FE211420FFF740FE33B030BD013311F8F5
:10572000012FE254F0E770B5B2B032AC0223054667
:1057300004F8C83D04F06AFEC72828BFC720064603
:105740000023681E9E420BDC06F13200FFF7C2FD0B
:105750002346721CFF211420FFF71EFE32B070BDDD
:10576000013310F8012FE254ECE700002DE9F04F6F
:105770000128B9B08146884603DC1B20FBF7EAFE0E
:1057800058E00868C2072BD4042829D9036803F01D
:105790000F03042B24D1FDF743FF0546D8F804007E
:1057A000C3071FD404281DD9036803F00F03042B7B
:1057B00018D1FDF735FF0646214BDFF890A01B6896
:1057C00003930027039BBB420EDC00962B461D4A29
:1057D000C82106A804F0A0FD06A8FFF7A4FFCCE7A7
:1057E000194DDBE7184EE7E70C2303FB07F202EB4A
:1057F0000A03294652F80A00049304F0FDFD049BB5
:10580000044618B9D3E9013B9C4201DB0137D9E7D3
:105810000BEBC40231465BF834000593049204F0AC
:10582000EBFDDDE9042340B9536808F10801A9F153
:105830000200984739B0BDE8F08F0134E4E700BFBB
:1058400034740120A4BF00001FB80000648D012043
:105850002DE9F0411F4F204AD7F80080054600236C
:10586000F02098450EDC0024F02000FB04F15318D2
:10587000565C8EB101340A2CF7D11848BDE8F041CE
:10588000FFF751BF00FB03F154186478AC4201D11B
:10589000515CE9B90133E4E7F0223146184604F0DF
:1058A00017FA0F49457051F8351085700222A0454E
:1058B0000270C0E90212C0E9046601DC01343C60F8
:1058C000002329461A461020BDE8F041FFF764BDC9
:1058D000BDE8F0819C0500206C7A0120EDC300003A
:1058E000CC83012070B5FFF78BFD094EFF246FF0CC
:1058F000070505FB046393F8FC37043B012B03D831
:10590000E043C0B2FFF7A4FF013CF2D170BD00BF7D
:10591000CC8301202DE9F8431D4E07460D46002497
:10592000B046E3009A191279062A01D0032A23D13E
:1059300058F80300836803F07F031C2B1CD1C36855
:1059400003F07F02042A17D1026902F07F02192AAC
:1059500012D11B0A00EB83001030FDF761FE0378C3
:10596000814633B104F052FDA84205D100239D4287
:1059700007DCE0B2FFF76CFF0134FF2CD1D1BDE8AA
:10598000F88319F80310FA5C9142F5D10133EEE780
:10599000CC830120F8B5094F0546FF246FF00706B8
:1059A00006FB047393F8FC37AB4203D1E043C0B26B
:1059B000FFF74EFF013CF3D1F8BD00BFCC830120BF
:1059C0002DE9F84FFDF750FB584B1A68824284BF0F
:1059D00000221A601A6842F20F71821A8A420BD9A9
:1059E0005349186000235A181279073A022A0FD92E
:1059F0000833B3F5FF6FF6D1BDE8F88F0720FFF746
:105A0000C9FF8AF800802EE00820FFF7C3FF3FE0BF
:105A1000FDF732FB002814BF044601240020FDF7E7
:105A200011FC81460020FDF721FC424D424E074605
:105A3000B9F1000F17D02B68002B70D133682C60A0
:105A4000002B6FD0DFF8F8B0DFF8F0A09BF8003043
:105A50004FF00108002BD1D10920FFF79BFF8AF8F6
:105A600000808BF80080AFB133689BB92B6834603D
:105A70001BB3DFF8C8B0DFF8C8A09BF800304FF0C8
:105A80000108002BC0D10920FFF784FF8BF80080AC
:105A90008AF800802B6883B1284A1178904661B952
:105AA0009C4238BF2C602B68E31A312B05D90720A4
:105AB000FFF770FF012388F80030326882B1204B75
:105AC0001978984661B9A24288BF34603368E41AF5
:105AD000312C05D90820FFF75DFF012388F800303D
:105AE0002B685BB1B9F1000F08D1144C227812B9C0
:105AF0000720FFF74FFF00232B6023703368002B34
:105B00003FF47AAF002F7FF477AF0D4C227812B9B3
:105B10000820FFF73FFF0023336023706CE7002F5E
:105B2000A2D1B9E7002FA1D1B4E700BF24700120B2
:105B3000CC830120147001201C70012018700120FA
:105B40002070012037B50546FFF75AFC02A8002453
:105B500040F8044DFDF75EFB21462046FEF7CAF9EA
:105B6000FEF744FCFDF796FBFDF75EFCFDF778FCC5
:105B7000FEF7D8FCFDF79CFA25B1FDF701FD0248C0
:105B8000FFF7D1FD03B030BDDEC3000000230146A6
:105B90001A461120FFF700BC07B513128DF801203B
:105BA0008DF802301314120E8DF800108DF80330AA
:105BB0008DF8042001466B4605221320FFF7ECFB0D
:105BC00003B05DF804FB0A4601461220FFF758BCFB
:105BD00070B50C46054601F13200FFF77BFB2B4602
:105BE000224600211B20BDE87040FFF7D5BB10B452
:105BF000144603460A46142021465DF8044BFFF77D
:105C0000CBBB000030B5084C01444FF0FF33884255
:105C100001D3D84330BD10F8015BDAB26A4054F8C2
:105C2000222082EA1323F2E7C0BF0000FE2837B526
:105C3000044614D80B4B53F8300080B1416808304B
:105C40008900FFF7DFFF02AD45F8040D0920FFF7DB
:105C500041FB2B46042221461720FFF79DFB03B092
:105C600030BD00BFCC830120F8B50746FEF7DCFD50
:105C70004FF0FF3504460CB92846F8BD2668C6F338
:105C80000743152B0CD104F10801384604F0B4FB8E
:105C900008B9C6F307252046FEF7C6FC0446EAE726
:105CA0001D2B08BF4FF0FF35F5E700002DE9F04749
:105CB000BF4CC04D9CB0FFF7F3FA2068C0F580617F
:105CC0002844FDF72BFC23680344064623607BB180
:105CD000B94F002E0FDC2B78FA2B40F0308123686F
:105CE000022B16DCFFF7C8FA10B10120FFF79CFA6F
:105CF0001CB0BDE8F0872068C0F580612844FDF73E
:105D00000DFC2368034406462360FDF7ADF93860B7
:105D1000DFE76878AC78831E182B00F20681DFE895
:105D200013F019002D003100350038004100040146
:105D30004B0080008A008E00A400E000F100040106
:105D4000040104010401040104010401040104012B
:105D50000401FF00FF2C0FD02046FFF7A3FC974A59
:105D6000002342F8343002EBC402214613711320A1
:105D700000931A46FEF740FE0320B7E72046FFF7E0
:105D800067FDF9E72046FFF78DFCF5E7FFF7AAFD71
:105D9000F2E7FFF735FB0020FFF7D4FE8848FFF756
:105DA000C2FCE9E7632CE7D8864B214653F8242050
:105DB0001520FFF765FBDFE7FEF736FD6FF00708FC
:105DC0000446002CD8D02768C7F30743152B04D00E
:105DD0002046FEF729FC0446F3E704F108063046A6
:105DE00004F014FB05460530FFF774FAFB20FFF7BB
:105DF0000DFA1D20FFF70AFAC7F30720FFF706FA8E
:105E0000E8B2FFF703FAC5F30720FFF7FFF9A8EBA5
:105E10000407F3199D42DBDD16F8010BFFF7F6F9D5
:105E2000F7E7002300931A4619461D20FEF7E4FD0C
:105E3000FDF7A6FBA0E72046FFF7F8FE9CE7FDF77D
:105E400023F9614A00906421604B03A804F064FACE
:105E5000022303A88DF80C3004F0D8FA03AB0246F5
:105E600000211620FFF798FA86E7544F002557F8CF
:105E7000354007EBC5035CB3D4F8048093F804A065
:105E80004FEA8806B01DFFF725FAFB20FFF7BEF9A1
:105E9000012006F10109FFF7B9F9E8B2FFF7B6F9F9
:105EA0005FFA89F0FFF7B2F9C9F30720FFF7AEF9FF
:105EB0005046FFF7ABF9083404EB0609A1450BD8AF
:105EC000FFF7EEF906EB080001F05CFCFFF7E8F9DC
:105ED0000135FF2DCBD14FE714F8010BFFF796F9F1
:105EE000ECE70024FFF78CFA224621460094234673
:105EF000DA20FEF781FD4FF4FF6221462F4803F0C0
:105F0000E7FE95E7012C02D1FEF7B6FB34E7022C41
:105F100002D1FEF76FFD2FE70120FFF713FE2BE7FD
:105F200000231A4621461A209CE7A0F1C803052B3E
:105F30003FF622AF00221146FBF744FA1CE7FB2B89
:105F40007FF4D3AE2268042A7FF7CCAEB5F8037095
:105F500040F2F6339F423FF7C8AE3B1D9A427FF7AF
:105F6000C1AEEB5CFE2B7FF4C0AE6878AC781B282A
:105F700007F1FF367AD02DD807285ED0082837D011
:105F800001282CD1FF2C11D02046FFF78BFB6D7917
:105F90000F4B00932146BB1E2A460A20FEF72CFD1C
:105FA000064B43F8340003EBC4042571781D9DE6CD
:105FB000387801203874012028700120CC8301201A
:105FC000C0C30000C48B0120D7C30000D2C30000AF
:105FD0003E7401201D285BD04DD31E2870D0A0F147
:105FE000C803052BE2D83F4A3146FBF7EBF9DDE762
:105FF000632CDBD86B79022B0CD0032B14D0012B34
:10600000D4D1D5F80630384A5B0043F0010342F89A
:106010002430CBE7002EC9DDB91E3448FDF71DFD45
:10602000314B43F82400C1E7AB79002B2E4B0CBF5A
:106030000022042243F82420B8E7632EB6DC32465F
:10604000284903A803F020FE1CAB1E4403A800232C
:1060500006F8643CFFF708FE0028A7DB224B214628
:1060600053F820201520FFF70BFA9FE731461D4813
:10607000FFF750FC9AE7FF2C98D06A79022A95D84E
:106080001A4B00932146BB1E0B20FEF7B5FC8DE793
:10609000632EA8BF6326002303A9B3420BDB1CAA0F
:1060A00026EAE6731344002203F8642C15200091BD
:1060B000731C2146E9E7EA185279CA540133ECE728
:1060C000012C7FF473AF002E7FF770AF6B791BB19B
:1060D000322BA8BF32231C4664235C43044B1C6054
:1060E00064E700BF3D740120C48B01203E74012091
:1060F00004000020084B01221A60084A1368002B94
:10610000FCD0074B1868042390FBF3F006384000DE
:1061100040F00100704700BF00C0004000C10040D7
:1061200008C500400120704710B5064C204600F01D
:106130008BFE0549204600F0EDFE044B01221A605B
:1061400010BD00BF74780120801A06003C78012041
:1061500010B5064C204600F077FE0549204600F0B9
:10616000D9FE044B01221A6010BD00BF3079012016
:10617000801A06004078012010B501210D20FCF79F
:1061800089FF094C01210E20FCF784FF00210F201C
:10619000FCF780FF204600F099FD20461021BDE865
:1061A000104000F0A9BD00BF547801202DE9F8434C
:1061B0000C68E30704D40D20BDE8F843FBF7CAB927
:1061C00064102FD4FCF764FFA0422BDB0021204693
:1061D000FCF760FF4FF4FA620121204601F00AFB50
:1061E00000B3DFF86C8000254FF001090027072677
:1061F0004FF47A720121204601F0FCFA90B1282870
:10620000C4BF09FA06F31F4316F1FF36F0D205F8B2
:1062100008700135052DE9D1012206210920FDF77D
:106220009BFB08B900200FE003460B2243F8042F24
:10623000064900F1180411F8012F520042F0010242
:1062400043F8042F9C42F6D1BDE8F883437801203F
:106250004478012010B50468E30704D40D20BDE89C
:106260001040FBF777B96410FF2C01D91720F6E72F
:10627000FFF782FFE1B2024800F061FD002010BD8F
:106280005478012008B5FFF777FF0021034800F09C
:1062900056FD400040F0010008BD00BF54780120C9
:1062A000274A82B001210023ADF80630C2F8F0156C
:1062B000C2F8001519461A0102F1804202F5E042C7
:1062C0000133082BC2F81415C2F81015F3D11C4B7A
:1062D0004FF4E062C3F818250422C3F81425C3F86C
:1062E00010250DF10602C3F82C260122C3F8302632
:1062F0001A60D3F80021002AFBD00022C3F8002145
:1063000001225A600E4B1A46D3F804110029FBD023
:106310000021C3F8041101219960D2F81431002B37
:10632000FBD00020C2F81401C2F80005BDF8063009
:106330001BB28342C8BFA3F50B70400002B0704788
:106340000070004008B5FFF7ABFF400040F00100CF
:1063500008BD0000024A03480A21FEF7CFBF00BF74
:1063600004C4000054C4000070B50668F10705D5E8
:106370004568EA0702D58468E30704D40D20BDE828
:106380007040FBF7E7B87610802E01D91520F6E7AC
:106390006D10FF2D01D91620F1E76410FF2C01D9F3
:1063A0001720ECE70A4B1B680BB9FFF7BDFEF1B2F3
:1063B000084800F02DFEE9B2064800F00DFDE1B2FC
:1063C000044800F009FD034800F08DFE002070BD78
:1063D0003C780120747801200C4B1B6870B5064690
:1063E0000D4614460BB9FFF7B3FEF1B2084800F0B2
:1063F0000FFEE9B2064800F0EFFCE1B2044800F0FD
:10640000EBFC0348BDE8704000F06DBE4078012011
:10641000307901200128F8B536DD0D68EA0733D55B
:106420001A4B4C681B686D100BB9FFF77DFEE9B283
:10643000174800F0EDFD14F001050DD0C4F347013D
:10644000134800F0C9FC124800F04DFE18B123209B
:10645000FBF780F80020F8BD042CF4D9236803F082
:106460000F03092BEFD154F8046F094F7610AE4299
:10647000E9DD54F8041FCB0704D5C1F347013846C2
:1064800000F0AAFC0135F2E70120E4E73C780120A6
:106490007478012038B50468E20702D54568EB0737
:1064A00004D40D20BDE83840FBF754B86410802CAC
:1064B00001D91520F6E76D10FF2D01D91620F1E75F
:1064C000124B1B680BB9FFF72FFEE4B221461048B0
:1064D00000F09EFDE9B20E4800F07EFC00210C4861
:1064E00000F0A0FD20B14042400040F0010038BD66
:1064F00001222146064800F088FD054800F063FCB3
:106500000028F1D0024800F061FCEDE73C78012062
:106510007478012038B5124B1B6804460D460BB940
:10652000FFF716FEE4B221460E4800F071FDE9B215
:106530000C4800F051FC0B4800F0D5FD08B140427A
:1065400038BD01222146074800F05FFD054800F0F4
:106550003AFC0028F4D00348BDE8384000F036BCCF
:106560004078012030790120F8B5354E354D376837
:1065700004466FB90D211D20FFF7CCFF5A2816D114
:1065800001222A702A211D20FFF726FF01233360F4
:1065900095F90030022B29D0032B44D0012B45D193
:1065A00021461D20FFF7B6FF4FF0FF3424E00F21F6
:1065B0001920FFF7AFFF332805D102232B705F228C
:1065C00020211920E0E70D211E20FFF7A3FFC72897
:1065D0000AD103233A462A211E202B70FFF7FCFE26
:1065E0001B222A211E20CFE72F70CFE7012C13D1C9
:1065F00029211920FFF78EFF7F28C8BFA0F58070E2
:106600006FF07E039842B8BF1846C82358437F23D3
:1066100090FBF3F06043F8BD032C0BD12B21192024
:10662000C0E72D21FBE721461E20BBE74FF0FF34DA
:106630000020EAE7052CF4D04FF0FF340020DFE71C
:106640004C7801202C00002008B50120FFF78CFFBA
:10665000400040F0010008BD08B50320FFF784FFAB
:10666000400040F0010008BD08B50520FFF77CFFA1
:10667000400040F0010008BD38B5104B1B6813B94D
:106680000120FFF771FF0120FFF76EFF0446032092
:10669000FFF76AFF05460520FFF766FF6D4304FB21
:1066A000045400FB004002F03FFF01F09FFB03F0A9
:1066B00055FA400040F0010038BD00BF4C78012081
:1066C0000128F8B535DD0F68FB0732D54D6815F0A8
:1066D00001062ED1042D2CD92B6803F00F03092BB2
:1066E00027D16C68144B64101B68202CA8BF202491
:1066F0000BB9FFF719FDC7F3470122460F480F4FAB
:1067000000F083FC0435A64211DA0C4800F05BFB74
:1067100018B9700040F00100F8BD384600F056FB93
:10672000400040F0010045F8040F0136EBE760003F
:10673000F0E70120F0E700BF3C78012074780120E9
:1067400000207047012070470020704700207047EC
:1067500001207047002070470020704700207047DC
:1067600000207047002070470020704700207047CD
:106770000020704700207047704770477047000046
:10678000024A03480E21FEF7B9BD00BFB8C400009D
:1067900028C500000246104601320378013B1F2B3A
:1067A000F9D9704708B5FFF7F5FF0378002B39D00A
:1067B000222B00F1010011D1037823B1222B00F12B
:1067C000010204D11046BDE80840FFF7E3BF5C2B8F
:1067D00002D1437803B1821C1046EDE73A2BF2D088
:1067E0002C2BF0D07B2B0BD1FFF7D4FF0378002BA1
:1067F000E9D07D2B01D10130E5E7FFF7D3FFF5E7C5
:106800005B2B10D00246104612F8013B002BDAD069
:10681000202BD8DD2C2B05D003F0DF015D2901D022
:10682000222BF0D108BDFFF7B5FF0378002BCAD0AB
:106830005D2BE0D0FFF7B6FFF7E708B5F0B1FFF743
:10684000A9FF0378222B1AD07B2B1AD05B2B1AD0EE
:10685000A3F13002092A05D92D2B05D14278303A0F
:10686000092A07D8032009E0742B0ED0662B0ED01E
:106870006E2B0ED0181C18BF0120404208BD04200A
:10688000FCE70220FAE70120F8E70520F6E70620FA
:10689000F4E70720F2E738B5FFF77CFF03782D2BEC
:1068A00011D101304FF0FF34431E00210A2501E0D1
:1068B00005FB012113F8012F303AD0B20928F7D98E
:1068C00004FB01F038BD0124EEE710B51446FFF7D4
:1068D00061FF0378222B02D000230B7010BD621ED3
:1068E00001300378222BF7D0002BF5D05C2B07D09A
:1068F000441C002AF0DD01F8013B013A2046F0E794
:106900004378622B00F1020409D0662B09D06E2B6C
:1069100009D0722B09D0742B08BF0923E9E708239B
:10692000E7E70C23E5E70A23E3E70D23E1E710B5EA
:106930000446FFF737FF0346A342184604D90278FE
:10694000202A03F1FF33F7D910BD08B590B10378C1
:1069500083B1FFF71FFF037803F0DF035D2B09D03E
:10696000FFF720FF03782C2B08BF0130BDE808405B
:10697000FFF710BF002008BD38B50D1E0DDD0378F0
:106980005B2B0AD10130FFF705FF0124A54205D09A
:10699000FFF7DBFF10B10134F8E7002038BD38B550
:1069A000154609B100230B70F8B10378E3B1FFF786
:1069B000F1FE03782C2B044603D10130FFF7EAFEE9
:1069C000044623787D2B0FD019B12A462046FFF7C5
:1069D0007CFF2046FFF7E6FE03783A2B05D1013015
:1069E000BDE83840FFF7D6BE002038BD2DE9F041A4
:1069F0000D469AB004462F789FB32E21284603F007
:106A0000EEFC804690B1461B303F092F13D8284634
:106A1000FFF741FF01462046FFF7AEFF044604B3EF
:106A2000B8F1000F1DD001363544E4E7284603F0E5
:106A3000EDFC0646E8E723787B2B11D1601C64222D
:106A400001A9FFF7ACFF044658B13246294601A818
:106A500003F0E4FC0028E2D02046FFF7A3FEEEE7B7
:106A6000002420461AB0BDE8F08138B50D1E04465A
:106A70001CDDFFF7E2FE012807D1601C012D00D1CB
:106A800038BDFFF762FF013DF8E702280ED1002272
:106A90001146601CFFF783FF012DF1D0FFF755FF72
:106AA00000221146FFF77BFF013DF5E70020E7E7F5
:106AB000F8B50C1E074615461E4613DDFFF7BDFE52
:106AC00002280FD132462946781CFFF768FF012CB7
:106AD00000D1F8BDFFF739FF32462946FFF75FFFC7
:106AE000013CF4E70020F4E710B50446C8B1FFF715
:106AF00051FE03787B2B0AD101300024002211467D
:106B0000FFF74DFF68B1FFF74DFE0134F6E75B2B51
:106B100006D101300024FFF718FF10B10134FAE765
:106B20000024204610BD002870B514DD0D68EB0769
:106B300011D56D10013DFDF777FE00264FF0FF34B3
:106B400060B916B3304603F061FC01463046BDE83B
:106B50007040FCF782BF4FF0FF35ECE70368C3F3EA
:106B60000742152A0BD1C3F307239C42B8BF1C462A
:106B70009D4201D100F10806FDF756FDE0E71D2A10
:106B800004BF00264FF0FF34F6E7601C400040F0E1
:106B9000010070BD10B508680C46FCF741FDFFF719
:106BA00063F80028A2BF034B626843F8202000204E
:106BB00010BD00BFC48B012008B50868FCF730FD8C
:106BC000FFF752F80028AABF024B012053F820001B
:106BD00008BD00BFC48B012008B50868FCF720FD84
:106BE000FFF742F80028ACBF0420002008BD0000D9
:106BF000024A03480421FEF781BB00BFB8C500006C
:106C0000B1C5000008B5FCF73DFCFCF7DDFCFEF764
:106C100089FB0448FEF787FDFDF748FFBDE8084003
:106C2000FEF760BE07C60000FCF7FCB838B50025CB
:106C3000057329B90B4B0C4A0C48232102F0B6FF0F
:106C400001600B4951F82220027151F82330837101
:106C50009DF8103051F8233043710223C3718560D1
:106C600038BD00BF1FC600007EC600002DC6000054
:106C7000DCC60000037B23B94373837303610123E4
:106C80000373704784B00DF1100C0CE90E009DF8F1
:106C90000810026800230129C2F80035039B12D0B6
:106CA0000BD303290CD0C2F85435019BC2F824350C
:106CB0000123C2F8003504B0704743F00203F2E745
:106CC00043F00403EFE743F00603ECE710B5FFF7EA
:106CD000D1FF03688279C3F808254279C3F80C25EF
:106CE0000279C3F81025034BBDE810400ECBFFF727
:106CF000C9BF00BF687801200A0611D43F2912D805
:106D00001F2913D80F2914D8072915D803298CBF98
:106D10004FF080434FF000430268C2F824357047BB
:106D20004FF00073F8E74FF08063F5E74FF0006332
:106D3000F2E74FF08053EFE74FF00053ECE70368C2
:106D4000C3F81C15D3F80821002AFBD0D3F8180586
:106D50000022C3F80821C0B27047000007B5094BF4
:106D600009490A484FF080421A6000229A600222C4
:106D70001A710F2300930E220D23FFF757FF03B064
:106D80005DF804FB68780120003000405478012051
:106D90002DE9F84380460D46174601EB02090C46E3
:106DA0004C45A4EB05060BD0D8F8003014F8011BB5
:106DB0001B68404698470028F2D13046BDE8F8836A
:106DC0003E46FAE77047203000F03CBA203000F031
:106DD0002BBA203000F03CBA38B5437F0D460BB9D2
:106DE000002038BD00F16804204600F039FA002880
:106DF000F6D12046294600F008FA0120F1E700000C
:106E00002DE9F0411E4600254FF47A73C0E9015385
:106E10000C4B044640F8203B8846174600F0ECF93E
:106E200004F1680000F0E8F99DF8183063769DF8E9
:106E30001C302676C4E90487A37665772046BDE832
:106E4000F08100BFC4C60000F0B5837E2E4C2F4DEC
:106E50000121C17654F82320437E54F8233012F0E8
:106E6000200F14BF2F464FF0A04702F01F0213F06F
:106E7000200F03F01F0308BF4FF0A04502F5E0729A
:106E800003F5E07340F20C6647F8226045F8236092
:106E900003694FF0CC72C3F8242503690622C3F8B6
:106EA0000025827E036954F82220C3F80825427E1B
:106EB000036954F82220C3F80C2590F91830144ABD
:106EC0005C0903F01F03994004F1600342F82310AA
:106ED00090F91830002BBDBF03F00F0302F6FC320F
:106EE000D2189B18B5BF40234022137683F80023A5
:106EF00090F918300122590903F01F0302FA03F335
:106F0000034A42F82130F0BDDCC600000003005007
:106F100000E100E0C37EA3B103690022C3F80025AD
:106F20000A4B99420ED90A4B994294BF4FF08061A7
:106F30004FF0C8610369C3F8241503690622C3F83A
:106F4000002570474FF0CC71F4E700BFA086010028
:106F500090D003002DE9F041044688461F461546AF
:106F6000002A50D000F12006304600F059F923697C
:106F7000C3F88885236901221A622369C3F834653E
:106F80002369C3F8385523691A602269D2F84C3155
:106F90001BB9D2F82431002BF8D00023C2F84C31B1
:106FA0002269D2F85C311BB9D2F82431002BF8D019
:106FB0000023C2F85C3122696FB9D2F8243153B989
:106FC0000123D3612369D3F84821002AFBD0002292
:106FD000C3F8482109E0012353612369D3F8042150
:106FE000002AFBD00022C3F804212369D3F824210E
:106FF00012B10022C3F824212369D3F83C0520668E
:10700000C0B2BDE8F0811046FBE70123FFF7A2BF45
:1070100010B5044680F8B010683000F001F9012383
:10702000637710BDF8B500234377036990F8B0206B
:10703000C3F88825036901261E62036900F168050B
:107040000446C3F8445528460F4600F0FBF8236970
:10705000C3F8480523699E602369D3F850211AB903
:10706000D3F82421002AF8D00022C3F85021284662
:1070700000F0E8F8236930B1D3F860211AB9D3F8E9
:107080002421002AF8D00022C3F8602123696FB9B7
:10709000D3F8242152B90122DA612369D3F84821B7
:1070A000002AFBD00022C3F8482109E001225A61DE
:1070B0002369D3F80421002AFBD00022C3F804215D
:1070C0002369D3F8240168B10022C3F8242123697D
:1070D000D3F8C404C3F8C404022803D004280CBFA6
:1070E00003200420F8BD0121FFF79CBF70B5436960
:1070F000D3F86421044692B10022012500F1200654
:10710000C3F864210577304600F08AF86369C3F854
:10711000346563694022C3F8382563691D63636978
:10712000D3F86821DAB10025C3F8685104F1680684
:10713000012363772577304600F072F8D4F8B43035
:1071400003B19847636965773046C3F8446500F03A
:1071500079F86369C3F84805636901225A63636972
:10716000D3F8042162B10022C3F80421237F3BB18C
:107170006369D3F83C05D4F8B830206603B198476A
:107180006369D3F8242152B10022C3F82421636932
:10719000D3F8D024C3F8D024636901225A6170BDAA
:1071A0000148FFF7A3BF00BF747801200148FFF733
:1071B0009DBF00BF3079012007B514231322CDE90C
:1071C00000320A4A0A4811460323FFF719FE4FF01E
:1071D00040221E231F21CDE9003106480423114619
:1071E000FFF70EFE03B05DF804FB00BF0030004067
:1071F000747801203079012008B54022002102F086
:1072000067FD0022C0E9102208BD026C10B5531CB6
:10721000446C03F03F039C421CBF8154036410BDC7
:107220000023C0E910337047D0E9102393421FBFF9
:10723000C25C013303F03F03436414BF10464FF0B8
:10724000FF307047D0E91030181A48BF40307047FF
:10725000D0E91023934214BFC05C4FF0FF30704759
:10726000036C406C013303F03F031B1A5842584132
:10727000704700000649074A074B9B1A03DD043B91
:10728000C858D050FBDC00F04DF8F9F7D9F80000F1
:1072900084CB00000000002034020020FEE7FEE75F
:1072A000FEE7FEE7FEE7FEE7FEE7FEE7FEE7FEE7B6
:1072B000094B1B78062B0CD1084B1B681A0708D109
:1072C000074B186800F0F000A0F130035842584115
:1072D00070470020704700BFE00F00F0E40F00F09F
:1072E000E80F00F00C4B1B78062B10D10B4B1B68E2
:1072F0001A070CD10A4B186800F0F003302B08D0A5
:1073000000F0E000A0F140035842584170470020CF
:1073100070470120704700BFE00F00F0E40F00F05D
:10732000E80F00F008B5FFF7C3FF10B14A4B4B4A16
:107330001A60FFF7D7FF28B1494B4A4A1B68C3F3CD
:1073400042331360FFF7B4FF20B1474AD36823F0FC
:107350008073D360FFF7C6FF40B14FF08043002237
:10736000C3F80C21C3F81021C3F83825FFF7A0FF9C
:1073700010B13E4B03221A60FFF79AFF40B13C4B1D
:1073800005221A6001229A6700229A603F225A6001
:10739000384B1B78062B50D1374B1B681B074CD141
:1073A000364B1B6803F0F003502B46D14FF0805250
:1073B000334BD2F80414C3F82015D2F80814C3F8DC
:1073C0002415D2F80C14C3F82815D2F81014C3F8F9
:1073D0002C15D2F81414C3F83015D2F81814C3F8C9
:1073E0003415D2F81C14C3F84015D2F82014C3F891
:1073F0004415D2F82414C3F84815D2F82814C3F859
:107400004C15D2F82C14C3F85015D2F83014C3F828
:107410005415D2F83414C3F86015D2F83814C3F8F0
:107420006415D2F83C14C3F86815D2F84014C3F8B8
:107430006C15D2F84424C3F87025124AD2F888306B
:1074400043F47003C2F88830BFF34F8FBFF36F8FE0
:107450000D4B0E4A1A6008BD74C007400DF0ADBA5E
:10746000440200103C050040F0ED00E0A0050040A3
:1074700010560040E00F00F0E40F00F0E80F00F0BD
:1074800000C0004000ED00E0300000200090D0037C
:107490000120704703681322DB69184770470369AE
:1074A000C3F81C150369D3F81C21002AFBD0002265
:1074B000C3F81C210120704710B490F95C30144CC3
:1074C00059090122203103F01F0302FA03F344F8A3
:1074D000213003695DF8044B0421C3F808130369E4
:1074E0005A600369DA6003690022C3F80025026963
:1074F0004FF0FF33C2F80C350269C2F81435026947
:10750000C2F8083502691430C2F81035FFF788BE9A
:1075100000E100E01430FFF795BE1430FFF798BE8D
:107520001430FFF781BE0000036990F85E2010B5AB
:10753000C3F80C25036990F85D20C3F8142590F872
:1075400061200369012A01BF90F85F40C3F810452C
:10755000036990F8604006BFC3F80845036900223C
:10756000B1F5966FC3F86C2569D9B1F5166F69D975
:10757000B1F5965F69D9B1F5165F68D9B1F5615F6C
:1075800067D9B1F5964F66D9B1F5E14F65D9B1F537
:10759000164F64D9B1F5614F64D9B1F5963F64D9FE
:1075A000B1F5E13F63D9B1F5613F63D9364B9942FB
:1075B00063D9B1F5E12F63D9B1F5612F94BF4FF0D5
:1075C00070634FF080530269C2F8243503690422C6
:1075D000C3F8002501690023C1F808310169C1F829
:1075E0001C31016901230B6001698B600169C1F8DD
:1075F000042390F95C20510902F01F02934060318E
:10760000224A42F8213090F95C30002BBDBF03F0D4
:107610000F0302F6FC32D2189B18B5BF602360221C
:10762000137683F8002390F95C300122590903F0A6
:107630001F0302FA03F3154A42F8213010BD4FF43C
:107640009E23C0E74FF41D23BDE7114BBBE7114B51
:10765000B9E7114BB7E7114BB5E7114BB3E74FF45F
:107660001D03B0E74FF46B03ADE70E4BABE74FF0F4
:10767000EB73A8E74FF06C73A5E74FF08063A2E7C8
:107680004FF0E8639FE700BF90D0030000E100E007
:1076900000B013000050270000F03A0000A04E0098
:1076A00000C0750000903A012DE9F0411E4600250A
:1076B0004FF47A73C0E901530D4B044640F8143B74
:1076C00017468846FFF798FD0A4AC4F8108084F8E8
:1076D0005C7052F8263084F85D309DF8183052F80E
:1076E000233084F85E3084F861502046BDE8F08194
:1076F00070C70000DCC6000010B50369D3F808218C
:1077000004464AB1D3F818151430C9B2FFF77DFD0D
:1077100023690022C3F8082110BD00000148FFF7CB
:10772000EBBF00BFEC79012007B5212300930222B3
:10773000222303490348FFF7B7FF03B05DF804FBBA
:1077400000200040EC79012008B102F08DBD7047A7
:107750000A4B19680A4B30B5D3F804050C060D0A1C
:1077600044EA00024FF47A712B46A2FB014501FB6B
:107770000355E00B40EA454030BD00BF507A012080
:107780000010014038B5044648B1FFF7E1FF054657
:1077900000F01AF8FFF7DCFF401BA042F8D338BD19
:1077A000074B0022C3F8042182B0D3F80431054A04
:1077B0000193019B13680133DBB2136002B0704781
:1077C00000100140507A01207047704708B500F062
:1077D0005FF8FFF7FAFF0120FFF7D4FFFFF712FA77
:1077E000034CFFF721FA002CFBD0AFF30080F8E741
:1077F00000000000134B53F8203010B503F01F03B6
:10780000114C0120002900FA03F010492368B3FB52
:10781000F1F3014602FB03F34FF00A02B3FBF2F36C
:1078200014BF024600220A4800F014F842F2107316
:1078300058434FF47A722368B3FBF2F3B0FBF3F0D2
:1078400010BD00BFDCC600003000002040420F0029
:107850001005005030B504680C40944206D1013B3D
:10786000002BF8D112E0013B002B0FD004680C4034
:107870009442F8D1002405680D40954204D10134AA
:107880009C42F8D1002002E0201C00E0181C30BD12
:107890000D4BE02283F811234FF40032C3F880210E
:1078A0001A604FF080430122C3F818259A6003F54F
:1078B00088330021C3F808150221C3F80413C3F864
:1078C00044131A60704700BF00E100E0014B1860EC
:1078D000704700BF48000020222837B50CD84B4B1A
:1078E00053F82030052B00F0828007D8032B12D0EC
:1078F0007BD8022B00F08180002074E01D2B78D013
:1079000003D81C2BF8D1052206E01E2B73D01F2BA9
:10791000F2D1082200E002223D4B196808296EDDF1
:107920000A296FDD0D29B5BF0C240E240223032381
:107930003848C0F8F0350123C0F80035002005466E
:10794000030103F1804303F5E04301300828C3F845
:107950001455C3F81055F3D12F4B18682F4B1B68E3
:1079600000021B0303F4805300F4E0601843294B2A
:10797000C3F81805C3F81425C3F810250DF1060245
:10798000C3F82C260122C3F830261A60D3F8002150
:10799000002AFBD00022C3F8002101225A601D4BAF
:1079A0001A46D3F804010028FBD00020C3F80401D4
:1079B00001209860D2F81431002BFBD00023C2F8CC
:1079C0001431BDF906209A42124AB8BFADF806300C
:1079D000A142C2F80035BDF9060004D035BF611AD6
:1079E000091BC840884003B030BD032294E704223D
:1079F00092E7062290E707228EE701228CE708240F
:107A0000002395E70A24012392E700BFDCC60000AB
:107A10004000002000700040440000205C7A0120FB
:107A2000222830B53CD8224B53F82000214B0022AD
:107A30001D4653F82240B4F1FF3F32D11E4C45F8A9
:107A400022006FEA41411D4D1D4B246853F822303E
:107A50006FEA514125F81210012101FA04F4C3F82C
:107A60006005013CC3F8640505EB4202C3F86805F4
:107A7000C3F86C050020C3F80015C3F80C05C3F863
:107A80000405C3F80845C3F81405C3F81005C3F886
:107A90002025C3F82415C3F82815C3F82C059960D0
:107AA00030BD8442CAD00132032AC2D1F8E700BFF8
:107AB000DCC600003400002048000020547A012079
:107AC00098C70000222815D8114B124A53F82030CD
:107AD00013F0200F08BF4FF0A04203F01F0303294B
:107AE00008D8DFE801F00210080C03F5E07300216C
:107AF00042F82310704703F5E0730C21F8E703F513
:107B0000E0730421F4E703F5E0730321F0E700BF1D
:107B1000DCC6000000030050222813D80A4B53F89B
:107B200020000A4B10F0200F4FF0010200F01F0060
:107B300008BF4FF0A043824011B9C3F80C2570472D
:107B4000C3F80825704700BFDCC6000000030050E2
:107B5000222810D8094B0A4A53F8203013F0200F7E
:107B600008BF4FF0A04203F01F03D2F81005D84021
:107B700000F0010070470020704700BFDCC6000025
:107B8000000300502DE9F04106460D4601EB0208C6
:107B90000C464445A4EB050707D0336814F8011BD5
:107BA0001B68304698470028F3D13846BDE8F0817D
:107BB0002DE9F041C1F30A57A7F2FF35132D82B02A
:107BC00002460B460C464FEAD178064633DC002DC0
:107BD0004EDB3B49294103EA0100104326D0490806
:107BE0000B4052EA03060CD04FF48023132D24EAF5
:107BF000010143FA05F444EA01040CBF4FF00046CA
:107C00000026304901EBC8082346D8E90045324632
:107C10002046294601F03CFBCDE9000122462B46D7
:107C2000DDE9000101F032FB02460B461046194621
:107C300002B0BDE8F081332D07DDB5F5806FF5D1D9
:107C400001F026FB02460B46F0E7A7F213474FF080
:107C5000FF31F9400842E9D049080842D1D04FF03D
:107C6000804320EA010143FA07F741EA0706C8E723
:107C700021F000410143D9D0C3F3130101434E4227
:107C8000104D0E43360B05EBC8055C0C06F40023C3
:107C9000D5E90067640443EA04010B4630463946DF
:107CA00001F0F6FACDE9000132463B46DDE900017C
:107CB00001F0ECFA21F00041024641EAC873B5E751
:107CC000FFFF0F00A8C70000F8B5C1F30A57A7F2DD
:107CD000FF35132D0A460B46044611DC002D2ADB26
:107CE0008C461F4929410A422BD04FF400232B41D7
:107CF000634423EA01030026344619462046F8BDB2
:107D0000332D05DDB5F5806F1ED011462046F8BD38
:107D1000A7F213474FF0FF3121FA07F73842F4D0AA
:107D20000122C5F1330502FA05F5461928BF9B1853
:107D300026EA0706E0E7013501F0004309D00026F6
:107D4000DAE70028D1D1E0E7024601F0A1FA0446C3
:107D5000DCE743F07F5343F440130026CCE700BF39
:107D6000FFFF0F0030B51F4A21F00043934287B058
:107D70001BDD1D4A934205DD02460B4601F086FAE3
:107D800007B030BD02AA00F08FF800F00300012810
:107D9000DDE9042311D002281BD098B1DDE90201EE
:107DA00000F062FB01F10041EAE7002300930022AA
:107DB000002301F09DF807B030BDDDE9020100F0BD
:107DC00053FBDDE70124DDE90201009401F090F8A6
:107DD000D6E70124DDE90201009401F089F801F100
:107DE0000041CDE7FB21E93FFFFFEF7F2DE9F04F99
:107DF0008BB004460D4600F075FA294B93F900A0AC
:107E0000BAF1FF3F06460F4612D022462B462046C7
:107E1000294601F08DFE834650B94FF000084FF01F
:107E2000000942464B462046294601F059FE20B93A
:107E3000304639460BB0BDE8F08F0122194BCDF822
:107E400020B00092CDE90445CDE902450193BAF195
:107E5000000F17D042464B464046494601F0F8FC19
:107E6000BAF1020FCDE906010ED101F0BDFE2123CA
:107E70000360089B73B9DDE90667304639460BB0ED
:107E8000BDE8F08FCDE90689684601F071F9002858
:107E9000EFD1EAE701F0A8FE089B0360EBE700BF23
:107EA0004C000020B8C700002DE9F04FC84E21F06B
:107EB0000047B7428FB00B4640F38F809246C54AC9
:107EC00097420C4626DC0029B7A3D3E9002340F3F0
:107ED0008F8001F0DBF9C04B9F4204460D4600F055
:107EE0004681B3A3D3E9002301F0D0F902460B4643
:107EF000CAE900232046294601F0C8F9ACA3D3E91A
:107F0000002301F0C3F90125CAE9020128460FB098
:107F1000BDE8F08FB14A974240F38980B04A97425A
:107F200000F31C813D15A5F21645A7EB0553194634
:107F30001F46064601F012FE01F0F6FA8046894619
:107F400002460B4630463946CDE9088901F09EF9D4
:107F50000022A44B01F052FB8946804601F0FEFD51
:107F600001F0E2FA02460B4606460F4640464946F5
:107F7000CDE90A6701F08AF900229A4B01F03EFB35
:107F800000220023CDE90C0101F0A0FD002800F043
:107F90005D81002330463946002201F097FD00281C
:107FA00014BF01230223904A019202212A46009124
:107FB00008A8514600F07CFB002C054614DADAF8DC
:107FC0000420DAF80C3002F1004203F1004345428C
:107FD000CAF80420CAF80C3006E0C2E90001002506
:107FE0000024C2E90245002528460FB0BDE8F08F05
:107FF00001F04EF9784B9F4204460D4600F008818F
:108000006BA3D3E9002301F043F902460B46CAE90A
:1080100000232946204601F039F965A3D3E900235E
:1080200001F036F94FF0FF35CAE90201DCE701F053
:1080300015F861A3D3E900238046894601F0DEFAF2
:1080400000226A4B01F024F901F088FD054601F099
:108050006BFA55A3D3E90023CDE9040101F0CEFA70
:1080600002460B464046494601F010F950A3D3E9B9
:108070000023CDE90201DDE9040101F0BFFA1F2D63
:108080008046894602460B46DDE9020140F3B08096
:1080900001F0FCF883460E463F15C6F30A53FB1A5F
:1080A000102B40F3B08046A3D3E90023DDE904019F
:1080B00001F0A4FA8046894602460B46DDE902013A
:1080C00001F0E4F802460B46DDE90201CDE90623A2
:1080D00001F0DCF842464B4601F0D8F83AA3D3E968
:1080E000002380468946DDE9040101F087FA424613
:1080F0004B4601F0CBF80B46024680468946DDE947
:10810000060101F0C3F8C1F30A53FF1A312F834669
:108110000E4600F39D8002460B46CAE90023DDE9C6
:108120000623CDE902235A463346DDE9020101F078
:10813000ADF842464B4601F0A9F8002C02460B462A
:10814000CAE90223BFF650AF06F1004601F1004133
:10815000CAE900B6CAE902016D4245E7024601F0EC
:1081600095F80025CAE90201CAE900013CE714A319
:10817000D3E9002301F08AF813A3D3E900230D46C5
:10818000044601F083F802460B46CAE9002329465B
:10819000204601F07BF80CA3D3E9002301F076F828
:1081A0000125CAE902011FE700004054FB21F93F05
:1081B0003163621A61B4D03D83C8C96D305FE43F5A
:1081C0000000601A61B4D03D7370032E8A19A33B7E
:1081D000FB21E93F7BD90240FB21F93FFB213941DB
:1081E000FFFFEF7F0000704140C800000000E03F4B
:1081F00001F04CF83A4B6A1E834653F82230BB42DA
:108200000E463FF449AF5A463346CAE900238AE78F
:108210002BA3D3E9002301F03BF82BA3D3E90023E0
:108220000D46044601F034F802460B46CAE9002325
:108230002946204601F02AF823A3D3E9002301F0C0
:1082400027F84FF0FF35CAE90201CDE60323AAE67D
:108250001FA3D3E90023DDE9040101F0CFF9DDE933
:10826000068906460F4602460B464046494601F03F
:108270000DF802460B4640464946CDE9022301F07F
:1082800005F832463B4601F001F813A3D3E9002379
:1082900006460F46DDE9040101F0B0F932463B46DF
:1082A00000F0F4FF02460B4680468946DDE90201F4
:1082B00000F0ECFF83460E46A5E700BFAFF3008059
:1082C0000000601A61B4D03D7370032E8A19A33B7D
:1082D0000000002E8A19A33BC14920259A837B39CF
:1082E000C0C700005F4A8A432DE9F0410D460746AA
:1082F00000F0948000290B460446064654DD0F1515
:1083000000F0A780C3F31303A7F2FF3743F48013F1
:10831000F20FF80702EB43034FEA460503D5ED0FD2
:1083200005EB4303B50000267F10B44616224FF438
:1083300000110CEB010098424FEAD5744FEA450555
:1083400003DC1B1A00EB010C0E44013A04EB43035F
:108350004FEA5101EDD11046964620244FF00042DD
:1083600009E052D05B00013C03EBD5734FEA5202A7
:108370004FEA450537D0634502EB0E01F1DD0029D8
:1083800001EB020E0ADBE046A3EB0C03A94288BF17
:1083900003F1FF336D1A1044C446E3E7BEF1000F4A
:1083A000F1DB0CF10108EFE721F00042024329D094
:1083B000002945D10146CA0A153B4905002AFAD0D1
:1083C00012F4801001D048E030465200D40200F18F
:1083D0000106F9D5C6F1200401FA06F6E1401F1A9C
:1083E00041EA02038EE72B4324D14408731003F1C2
:1083F0007F53F20703F5001348BF44F0004403EB3A
:10840000075127463846BDE8F081A942AAD800297D
:1084100001EB020EC2DB98460023BBE702460B4687
:1084200001F0ECF83A462B4600F032FF074638469A
:10843000BDE8F081411C16BF421C01365408D5E747
:10844000024600F023FF02460B4601F001FA074600
:10845000D8E71A4621463B46B2E70E4620244FF0A5
:10846000FF30BBE70000F07F2DE9F04F21F0004620
:10847000B6F1795F85B00C4692469B4605466BDAAD
:1084800001F06CFB002800F0E2802A4623462846D3
:10849000214601F0B3F874A3D3E90023804689464E
:1084A00001F0ACF872A3D3E9002300F0F1FE4246DC
:1084B0004B4601F0A3F870A3D3E9002300F0E6FED9
:1084C00042464B4601F09AF86DA3D3E9002300F031
:1084D000DFFE42464B4601F091F86BA3D3E900233F
:1084E00000F0D4FE42464B4601F088F868A3D3E979
:1084F000002300F0CDFE42464B4601F07FF8CDE967
:1085000000010022644B4046494601F077F8DDE95E
:10851000002306460F464046494601F06FF8524692
:10852000804689465B462846214601F067F80246A8
:108530000B464046494600F0A9FE02460B4630462F
:10854000394600F0A3FE02460B460020534900F0D6
:108550009DFE05B0BDE8F08F02460B4601F04EF8D7
:1085600041A3D3E900238046894601F047F840A3A0
:10857000D3E9002300F08CFE42464B4601F03EF862
:108580003DA3D3E9002300F081FE42464B4601F0B3
:1085900035F83BA3D3E9002300F07AFE42464B4670
:1085A00001F02CF838A3D3E9002300F06FFE424617
:1085B0004B4601F023F836A3D3E9002300F068FE10
:1085C0004B46424601F01AF8354B9E42CDE9000178
:1085D00097DD344B9E424FF000023DDCA6F50013C0
:1085E00000202E4916461F4600F050FECDE902013C
:1085F0000022294B4046494601F000F832463B46EE
:1086000000F044FEDDE9002306460F464046494699
:1086100000F0F4FF5246804689465B4628462146D4
:1086200000F0ECFF02460B464046494600F02EFEA5
:1086300002460B463046394600F028FE02460B46FD
:10864000DDE9020100F022FE05B0BDE8F08F13491C
:10865000002005B0BDE8F08F134B144FCDE9022385
:108660000026C5E7AFF30080D43888BEE9FAA8BD7C
:10867000C4B1B4BD9EEE213EAD529C804F7E923E71
:108680009015CB19A001FA3E7751C1166CC1563F27
:108690004C5555555555A53F0000E03F0000F03FB3
:1086A0003233D33F0000E93F0000E73F0000D23FF4
:1086B0002DE9F04FADF5197DBE4CA29EBE4D54F88C
:1086C00026700793D41E85FB0465E417C4EBA5044C
:1086D00024EAE4741D46631CA3EB8303013D02EB13
:1086E000C30305937B1909940497019506460B91E2
:1086F000A4EB05041BD423445D1C20AF4FF00008FD
:108700004FF00009DDF88CA208E05AF8240000F0D0
:108710000BFF0134AC42E7E8020108D0002CF4DA88
:10872000013440464946AC42E7E80201F6D1049BD9
:10873000002BC0F2B083079BA6F10802DB001146B4
:10874000039220AA02EB0309029301EB0308049BA6
:1087500072AA02EBC30B0DF5E07A019B002BC0F26D
:108760009581039C4D460026002775E90223F4E914
:10877000020100F043FF02460B463046394600F046
:1087800087FD444506460F46EFD1EAE80267DA4521
:1087900009F10809E1D1DDE90204049920448B00C4
:1087A00082460BA8A3F10802C31808930CAB13442C
:1087B0000A938B4698AB03EBCB03BBF1000F53E955
:1087C000284529DD70AB03EBCB080DF13009002201
:1087D0007A4B2046294600F011FF01F0BFF900F066
:1087E000A3FE0022764B06460F4600F007FF024626
:1087F0000B462046294600F049FD01F0AFF978E923
:10880000022349F8040B3946304600F041FD70ABB5
:10881000984504460D46DAD1DDF8149020462946E5
:108820004A4600F0A9FC00224FF07F5304460D4653
:1088300000F0E4FE00F018FC0022624B00F0DEFEC7
:1088400002460B462046294600F020FD0D46044610
:1088500001F084F9804600F067FE0B460246294687
:10886000204600F013FD4B46002B06460F4640F312
:10887000E1800BF1FF320CA9C9F1180351F8225025
:1088800045FA03F101FA03F30CA8EB1A40F8223081
:10889000C9F11705884443FA05F5002D2CDDBBF11D
:1088A000000F08F1010840F394820C9C002C40F06A
:1088B000A780BBF1010F0AD00CA9012251F8044F87
:1088C000531C002C40F09E809B451A46F6D1059B18
:1088D000002B0EDD012B00F09C81022B09D10BF146
:1088E000FF320CAB0CA953F82230C3F3150341F847
:1088F0002230022D00F0AF8000220023304639469E
:1089000001F0E4F8002800F06682049B0BF1FF39C7
:108910004B4510DC0BF180430CAA013B089802EB9D
:108920008303002253F80419834242EA0102F9D179
:10893000002A40F0B580049B0CAA013B52F823307A
:10894000002B40F0A1800A9A012352F80419013348
:108950000029FAD05B440BF101099945069349DCE3
:10896000099A079909EB020801EB0B0508F1804809
:1089700002EB030BA39B08F1FF3803EB880870ABF5
:1089800003EBC909A39B20A903EB8B0301EBC505EE
:10899000029358F8040F00F0C7FD019B002BC5E9B6
:1089A000000105F1080B28DB083D039C0026002789
:1089B0000CE000BF88C90000ABAAAA2A0000703EE4
:1089C000000070410000204075E80201F4E9022334
:1089D00000F014FE02460B463046394600F058FCC3
:1089E000544506460F46EFD1029B9845E9E80267D9
:1089F0005D46CED1DDF818B0DCE600260027F3E7AF
:108A0000012300220CA9C4F180749B4541F8224047
:108A10000EDD51F8232001EB8B0001EB83036FF097
:108A20007F4100E01A688A1A43F8042B8342F9D187
:108A300001244CE706D10BF1FF330CAA52F8235066
:108A4000ED152AE70022BE4B01F05EF8002840F049
:108A5000B981054650E732463B460020B94900F04F
:108A600015FC06460F46002C3FF446AF059AB54963
:108A7000002000F081FB02460B463046394600F0EC
:108A800005FC06460F4637E7012363E7002600276B
:108A9000EAE80267DA4509F108097FF45EAE7AE692
:108AA0000CAB059A53F82930183ACDE906850592A2
:108AB0006BB909F18043013B0CA901EB830353F827
:108AC000041909F1FF39183A0029F8D00592059ADE
:108AD0009C49002000F050FBB9F1000F04460D4600
:108AE000C0F2E0814FEAC90370AA02EB03080893C1
:108AF0000CAB03EB8906DFF850B208F10807043627
:108B00004FF0000A56F8040D00F00EFD22462B46E9
:108B100000F074FD5B4667E9020152462046294693
:108B200000F06CFD0CAB9E4204460D46EAD148AB0A
:108B300003930193CDF8149009F10103DDF810902F
:108B40000293C3464FF0000AB9F1000FC0F237811B
:108B5000DFF8F8815D4678A3D3E9002300260027DB
:108B6000002403E0544510DCF8E80223F5E8020194
:108B700000F044FD02460B463046394600F088FBC3
:108B80000134A14506460F46ECDA019BE3E8026793
:108B90000193029B0AF1010A9A45ABF1080BD3D16C
:108BA000A29BDDF81490032B2CD8DFE813F0E8002B
:108BB000D300D3003F00079B00200146002B40F06C
:108BC00043810D460B460B990446C1E900450399C4
:108BD0000246D1E9000100F059FBB9F1000F0CDDAC
:108BE000039D0124F5E90223013400F051FBA14566
:108BF000F8DA079B002B40F037810B460B990246B1
:108C0000C1E90223069B03F007000DF5197DBDE8BD
:108C1000F08F0BF1FF320CAB0CA953F82230C3F3E9
:108C2000160341F8223064E648AB0393B9F1000F14
:108C300040F35581039ACDF808904FEAC90302EB3F
:108C40000308D8E900AB0193914658E90267524600
:108C50005B463046394600F01BFB04460D46024693
:108C60000B463046394600F011FB52465B4600F099
:108C70000FFBC8E9000168E90245C145A246AB46C1
:108C8000E3D1DDF80890B9F1010F40F32881019B91
:108C9000039A1344D3E9006701939A460DF5947B38
:108CA0005AE9028932463B464046494600F0F0FA0E
:108CB00004460D4602460B464046494600F0E6FA99
:108CC00032463B4600F0E4FACAE900016AE902458F
:108CD000D34526462F46E3D10399019C002301F199
:108CE0001005083419461E46304674E9022300F088
:108CF000CFFAA5420346F6D10A460399D1E9008C82
:108D0000D1E902E90799002900F0B1800B9C2361A9
:108D1000069BC4F800800CF1004009F1004102F10B
:108D20000042606003F00700E1606261C4F808E09F
:108D30000DF5197DBDE8F08F00000040FB21F93FE3
:108D40000000E03F0000F03F0000703E50C900000E
:108D500048AB0393B9F1000FFFF62DAF039F00203E
:108D600007EBC9060836014676E9022300F090FABF
:108D7000B742F9D1079B002B3FF423AF64E0089C76
:108D8000039D083400222C4411461646304674E9EF
:108D9000022300F07DFAA5420246F6D10B46079960
:108DA00009B103F1004319460B9B1046C3E90001CA
:108DB000069B03F007000DF5197DBDE8F08F002636
:108DC0000027E2E6BBF1000F08F101087DDD022576
:108DD0006BE500247BE5CDE90685059D30463946E7
:108DE0006A4200F0C9F900223E4B06460F4600F0E9
:108DF0008BFE00B300223C4B3046394600F0FEFBB0
:108E000000F0ACFE044600F08FFB0022354B00F072
:108E1000F5FB0B4602463946304600F037FA00F0C3
:108E20009DFE0BF101090CAB183543F82B0005959D
:108E300043F829404BE63046394600F08FFE0CAB34
:108E4000D94643F82B0042E60B9C0B4601F100414A
:108E5000C4E9000103990246D1E9000100F016FAC5
:108E6000B9F1000F3FF7BCAE01F10041C5E618466D
:108E70000B9B4646744667464D461146C3E90401BE
:108E8000C3E90067C3E90245069B03F007000DF53F
:108E9000197DBDE8F08FA6F108030393079BDB0063
:108EA000029378E4A29B032B3FF6ACAE01A252F8EA
:108EB00023F000BFC58E0000518D0000518D0000D1
:108EC000298C00000022134669E732463B46002009
:108ED000064900F0DBF9022506460F460CE50023A3
:108EE0001A460AE7000070410000703E0000F03FA3
:108EF0002DE9F04F21F00046B6F1795F85B00C46C0
:108F000090469946054604DA00F028FE002800F055
:108F100085802A4623462846214600F06FFB0646F8
:108F20000F4602460B462846214600F067FB3EA34B
:108F3000D3E9002382468B463046394600F05EFB7B
:108F40003BA3D3E9002300F0A1F932463B4600F0F1
:108F500055FB39A3D3E9002300F09AF932463B468A
:108F600000F04CFB36A3D3E9002300F08FF9324622
:108F70003B4600F043FB34A3D3E9002300F088F91B
:108F80000E9BCDE900019BB30022334B404649467E
:108F900000F034FBDDE90023CDE9020150465946DB
:108FA00000F02CFB02460B46DDE9020100F06EF9F1
:108FB00032463B4600F022FB42464B4600F066F943
:108FC00023A3D3E9002306460F465046594600F036
:108FD00015FB02460B463046394600F059F9024669
:108FE0000B462846214600F051F905B0BDE8F08F48
:108FF00002460B463046394600F000FB14A3D3E985
:10900000002300F043F952465B4600F0F7FA2A4687
:10901000234600F03DF905B0BDE8F08F2846214613
:1090200005B0BDE8F08F00BF7CD5CF5A3AD9E53DF9
:10903000EB9C2B8AE6E55A3E7DFEB157E31DC73E09
:10904000D561C119A0012A3FA6F810111111813F65
:10905000495555555555C53F0000E03F21F00043A7
:109060001946704700000000C1F30A522DE9F84389
:10907000A2F2FF36132E0B460D46044688460746DD
:109080001DDC002E3DDB384A42FA06F901EA0902EE
:10909000024319D032A3D3E9002300F0F9F80022EB
:1090A000002300F03BFDD0B3002D04DA4FF4801311
:1090B00043FA06F6B04428EA090500272FE0332ECC
:1090C00006DDB6F5806F2FD019462046BDE8F8833F
:1090D000A2F213424FF0FF3929FA02F919EA000F00
:1090E000F2D01FA3D3E9002300F0D2F8002200231E
:1090F00000F014FD98B1002D24DB27EA090745464E
:109100000DE017A3D3E9002300F0C2F800220023EA
:1091100000F004FD18B1002D0BDB00273D463C4656
:1091200029462046BDE8F883024600F0B1F804461F
:10913000CBE725F000430D4A1F43002F18BF15460B
:109140000027ECE7142E08D00123C6F1340603FAF9
:1091500006F6371928BF9844CFE705F10108CCE798
:109160009C7500883CE4377EFFFF0F000000F0BFD5
:109170000020704700000000F8B5C1F30A53044610
:109180000D460E4617460BBB21F0004603463343FF
:109190001BD0354B002200F031FA344B9F4204467D
:1091A0000D4635DBC1F30A530E46363B3B4440F2D5
:1091B000FE72934232DC002B11DD26F0FF4626F4CE
:1091C000E00646EA035520462946F8BD40F2FF7204
:1091D0009342EBD102460B4600F05AF8F8BD13F16A
:1091E000350F28DA4CF250339F4222462B460ADDD7
:1091F00019A1D1E9000100F03DF817A3D3E900233C
:1092000000F0FCF9F8BD16A1D1E9000100F032F838
:1092100013A3D3E9002300F0F1F9F8BD22462B4651
:109220000DA1D1E9000100F025F80BA3D3E900233B
:1092300000F0E4F9F8BD26F0FF4626F4E0063633E8
:1092400046EA0355204629460022094B00F0D6F98C
:10925000F8BD00BFAFF300809C7500883CE4377E0A
:1092600059F3F8C21F6EA50100005043B03CFFFF48
:109270000000903C03F0004321F0004242EA030169
:10928000704700BF81F0004102E000BF83F000435F
:1092900030B54FEA41044FEA430594EA050F08BF91
:1092A00090EA020F1FBF54EA000C55EA020C7FEA55
:1092B000645C7FEA655C00F0E2804FEA5454D4EBD2
:1092C0005555B8BF6D420CDD2C4480EA020281EA9C
:1092D000030382EA000083EA010180EA020281EAD4
:1092E0000303362D88BF30BD11F0004F4FEA013126
:1092F0004FF4801C4CEA113102D0404261EB410135
:1093000013F0004F4FEA03334CEA133302D05242BA
:1093100063EB430394EA050F00F0A780A4F1010476
:10932000D5F1200E0DDB02FA0EFC22FA05F28018B0
:1093300041F1000103FA0EF2801843FA05F3594196
:109340000EE0A5F120050EF1200E012A03FA0EFC15
:1093500028BF4CF0020C43FA05F3C01851EBE3713F
:1093600001F0004507D54FF0000EDCF1000C7EEB5C
:1093700000006EEB0101B1F5801F1BD3B1F5001F9A
:109380000CD349085FEA30004FEA3C0C04F10104B9
:109390004FEA445212F5800F80F09A80BCF1004FE2
:1093A00008BF5FEA500C50F1000041EB045141EA64
:1093B000050130BD5FEA4C0C404141EB010111F465
:1093C000801FA4F10104E9D191F0000F04BF014610
:1093D0000020B1FA81F308BF2033A3F10B03B3F1EE
:1093E00020020CDA0C3208DD02F1140CC2F10C027E
:1093F00001FA0CF021FA02F10CE002F11402D8BFDC
:10940000C2F1200C01FA02F120FA0CFCDCBF41EAA7
:109410000C019040E41AA2BF01EB0451294330BD76
:109420006FEA04041F3C1CDA0C340EDC04F1140453
:10943000C4F1200220FA04F001FA02F340EA03002A
:1094400021FA04F345EA030130BDC4F10C04C4F170
:10945000200220FA02F001FA04F340EA0300294650
:1094600030BD21FA04F0294630BD94F0000F83F49A
:10947000801306BF81F480110134013D4EE77FEA7D
:10948000645C18BF7FEA655C29D094EA050F08BFC9
:1094900090EA020F05D054EA000C04BF19461046AA
:1094A00030BD91EA030F1EBF0021002030BD5FEAEE
:1094B000545C05D14000494128BF41F0004130BD16
:1094C00014F580043CBF01F5801130BD01F000456A
:1094D00045F0FE4141F470014FF0000030BD7FEADD
:1094E000645C1ABF194610467FEA655C1CBF0B46D8
:1094F000024650EA013406BF52EA033591EA030FEF
:1095000041F4002130BD00BF90F0000F04BF0021E6
:10951000704730B54FF4806404F132044FF0000519
:109520004FF0000150E700BF90F0000F04BF002192
:10953000704730B54FF4806404F1320410F00045F8
:1095400048BF40424FF000013EE700BF42004FEAF3
:10955000E2014FEA31014FEA02701FBF12F07F4370
:1095600093F07F4F81F06051704732F07F4208BF27
:10957000704793F07F4F04BF41F40021704730B52E
:109580004FF4607401F0004521F000411CE700BF7A
:1095900050EA010208BF704730B54FF000050AE0FD
:1095A00050EA010208BF704730B511F0004502D5FE
:1095B000404261EB41014FF4806404F132045FEA00
:1095C000915C3FF4D8AE4FF003025FEADC0C18BFA9
:1095D00003325FEADC0C18BF033202EBDC02C2F19B
:1095E000200300FA03FC20FA02F001FA03FE40EA2D
:1095F0000E0021FA02F11444BDE600BF70B54FF031
:10960000FF0C4CF4E06C1CEA11541DBF1CEA13550E
:1096100094EA0C0F95EA0C0F00F0DEF82C4481EA76
:10962000030621EA4C5123EA4C5350EA013518BF96
:1096300052EA033541F4801143F4801338D0A0FB83
:1096400002CE4FF00005E1FB02E506F00042E0FB30
:1096500003E54FF00006E1FB03569CF0000F18BF36
:109660004EF0010EA4F1FF04B6F5007F64F54074DE
:1096700004D25FEA4E0E6D4146EB060642EAC62171
:1096800041EA55514FEAC52040EA5E504FEACE2EDE
:10969000B4F1FD0C88BFBCF5E06F1ED8BEF1004FE1
:1096A00008BF5FEA500E50F1000041EB045170BD5D
:1096B00006F0004646EA010140EA020081EA0301A1
:1096C000B4EB5C04C2BFD4EB0C0541EA045170BD9D
:1096D00041F480114FF0000E013C00F3AB8014F117
:1096E000360FDEBF002001F0004170BDC4F1000460
:1096F000203C35DA0C341BDC04F11404C4F12005E1
:1097000000FA05F320FA04F001FA05F240EA02003B
:1097100001F0004221F0004110EBD37021FA04F671
:1097200042EB06015EEA430E08BF20EAD37070BD2B
:10973000C4F10C04C4F1200500FA04F320FA05F08A
:1097400001FA04F240EA020001F0004110EBD3708C
:1097500041F100015EEA430E08BF20EAD37070BDFC
:10976000C4F1200500FA05F24EEA020E20FA04F3D5
:1097700001FA05F243EA020321FA04F001F0004184
:1097800021FA04F220EA020000EBD3705EEA430EF5
:1097900008BF20EAD37070BD94F0000F0FD101F024
:1097A0000046400041EB010111F4801F08BF013C5D
:1097B000F7D041EA060195F0000F18BF704703F09B
:1097C0000046520043EB030313F4801F08BF013D22
:1097D000F7D043EA0603704794EA0C0F0CEA1355DE
:1097E00018BF95EA0C0F0CD050EA410618BF52EA98
:1097F0004306D1D181EA030101F000414FF000009E
:1098000070BD50EA410606BF1046194652EA4306AB
:1098100019D094EA0C0F02D150EA013613D195EA1F
:109820000C0F05D152EA03361CBF104619460AD167
:1098300081EA030101F0004141F0FE4141F4700171
:109840004FF0000070BD41F0FE4141F4780170BD61
:1098500070B54FF0FF0C4CF4E06C1CEA11541DBFC6
:109860001CEA135594EA0C0F95EA0C0F00F0A7F8C8
:10987000A4EB050481EA030E52EA03354FEA0131F5
:1098800000F088804FEA03334FF0805545EA131308
:1098900043EA12634FEA022245EA111545EA1065D0
:1098A0004FEA00260EF000419D4208BF964244F167
:1098B000FD0404F5407402D25B084FEA3202B61A86
:1098C00065EB03055B084FEA32024FF480104FF45A
:1098D000002CB6EB020E75EB030E22BFB61A7546CE
:1098E00040EA0C005B084FEA3202B6EB020E75EB61
:1098F000030E22BFB61A754640EA5C005B084FEAC9
:109900003202B6EB020E75EB030E22BFB61A754695
:1099100040EA9C005B084FEA3202B6EB020E75EBA0
:10992000030E22BFB61A754640EADC0055EA060E61
:1099300018D04FEA051545EA16754FEA06164FEAA4
:10994000C30343EA52734FEAC2025FEA1C1CC0D150
:1099500011F4801F0BD141EA00014FF000004FF0DD
:10996000004CB6E711F4801F04BF01430020B4F19E
:10997000FD0C88BFBCF5E06F3FF6AFAEB5EB030C56
:1099800004BFB6EB020C5FEA500C50F1000041EB53
:10999000045170BD0EF0004E4EEA113114EB5C0420
:1099A000C2BFD4EB0C0541EA045170BD41F48011F3
:1099B0004FF0000E013C90E645EA060E8DE60CEAFB
:1099C000135594EA0C0F08BF95EA0C0F3FF43BAF18
:1099D00094EA0C0F0AD150EA01347FF434AF95EACF
:1099E0000C0F7FF425AF104619462CE795EA0C0FB3
:1099F00006D152EA03353FF4FDAE1046194622E780
:109A000050EA410618BF52EA43067FF4C5AE50EA59
:109A100041047FF40DAF52EA43057FF4EBAE12E749
:109A20004FF0FF3C06E000BF4FF0010C02E000BF2A
:109A30004FF0010C4DF804CD4FEA410C7FEA6C5C0D
:109A40004FEA430C18BF7FEA6C5C1BD001B050EAB0
:109A5000410C0CBF52EA430C91EA030F02BF90EA9B
:109A6000020F0020704710F1000F91EA030F58BF5A
:109A7000994208BF90422CBFD8176FEAE37040F0BC
:109A8000010070474FEA410C7FEA6C5C02D150EA5A
:109A9000013C07D14FEA430C7FEA6C5CD6D152EA15
:109AA000033CD3D05DF8040B704700BF84461046DA
:109AB00062468C461946634600E000BF01B5FFF7D9
:109AC000B7FF002848BF10F1000F01BD4DF808EDA9
:109AD000FFF7F4FF0CBF012000205DF808FB00BF7A
:109AE0004DF808EDFFF7EAFF34BF012000205DF8D4
:109AF00008FB00BF4DF808EDFFF7E0FF94BF012021
:109B000000205DF808FB00BF4DF808EDFFF7CEFF21
:109B100094BF012000205DF808FB00BF4DF808ED60
:109B2000FFF7C4FF34BF012000205DF808FB00BF31
:109B30004FEA410C7FEA6C5C02D150EA013C0AD149
:109B40004FEA430C7FEA6C5C02D152EA033C02D13B
:109B50004FF0000070474FF0010070474FEA41029C
:109B600012F5001215D211D56FF47873B3EB62526F
:109B700012D94FEAC12343F0004343EA505311F096
:109B8000004F23FA02F018BF404270474FF0000028
:109B9000704750EA013005D111F0004008BF6FF066
:109BA000004070474FF00000704700BF1FB51C46D3
:109BB000094B1B680546D86852B1084B0091CDE9A6
:109BC000013207492B46224600F028F800F0B8FD84
:109BD000044B1A46F2E700BF5000002098C900006D
:109BE000A5C900001FB80000014B1868704700BFEE
:109BF0005000002008B5074B044613B10021AFF315
:109C00000080054B1868836A03B19847204601F02D
:109C100071FB00BF00000000D4C900000EB403B502
:109C2000014603AB054853F8042B0068019300F08C
:109C30007FF802B05DF804EB03B0704750000020DD
:109C400070B50D4E0D4CA41BA4100025A54209D1E2
:109C50000B4E0C4C01F050FBA41BA4100025A54298
:109C600005D170BD56F8253098470135EEE756F816
:109C7000253098470135F2E720020020200200201D
:109C8000200200203002002010B5431E0A449142F9
:109C900000D110BD11F8014B03F8014FF7E78842DE
:109CA00010B501EB020307D8421E99420AD011F801
:109CB000014B02F8014FF8E78342F5D98118D21A17
:109CC000D34200D110BD13F8014D01F8014DF7E763
:109CD00002440346934200D1704703F8011BF9E7A1
:109CE0009368013B002B10B4936007DA9469A34298
:109CF00001DB0A2902D110BC00F062BC1368581CB9
:109D000010601970084610BC7047F8B506460F463B
:109D10001446D518AC4201D1002007E03A4614F8A9
:109D2000011B3046FFF7DCFF431CF3D1F8BD0000F8
:109D30002DE9F04F9DB00C4617460393064618B127
:109D400083690BB900F0F4FD7B4B9C4257D17468DA
:109D5000A38918075DD52369002B5AD000230993E6
:109D600020238DF8293030238DF82A304FF0010B55
:109D7000B846454615F8013B0BB1252B54D1B8EB3D
:109D8000070A0BD053463A4621463046FFF7BDFF3F
:109D9000013000F0C280099B5344099398F80030C9
:109DA000002B00F0BA8000234FF0FF32CDE90523ED
:109DB000049307938DF853301A93A846052218F898
:109DC000011B5E4800F0C4FE049B78BBD90644BF6B
:109DD00020228DF853201A0744BF2B228DF85320E0
:109DE0002A782A2A2AD0079AA84600200A2541461E
:109DF00011F8013B303B092B69D960B324E0504B8B
:109E00009C4201D1B468A3E74E4B9C4208BFF46862
:109E10009EE72146304600F025FC00289ED04FF0FA
:109E2000FF301DB0BDE8F08FA846A2E7434A801A74
:109E30000BFA00F0184304904546BEE7039A111D43
:109E400012680391002A01DB079204E0524243F0BA
:109E500002030792049398F800302E2B0ED198F845
:109E600001302A2B38D1039B1A1D1B680392002B4B
:109E7000B8BF4FF0FF3308F102080593324D98F850
:109E800000100322284600F063FE40B14023401B2F
:109E900003FA00F0049B034308F10108049398F8C7
:109EA00000102A488DF82810062208F1010700F05A
:109EB0004FFE002837D0264B1BBB039B073323F0F4
:109EC000070308330393099B4B44099350E705FBB1
:109ED0000232012088468AE7002308F10108059331
:109EE00019460A25404610F8012B303A092A03D9B1
:109EF000002BC3D00591C1E705FB0121012380465A
:109F0000F0E703AB00932246124B04A93046AFF3AF
:109F10000080B0F1FF3F8146D5D1A3895B063FF5B4
:109F20007EAF09987DE703AB00932246094B04A955
:109F3000304600F087F8ECE72CCA0000D8C90000D2
:109F40004CCA00000CCA0000DEC90000E2C90000D3
:109F5000000000000B9D00002DE9F04791461F46D0
:109F60008A680B69DDF820809342B8BF1346C9F8B0
:109F7000003091F8432006460C4612B10133C9F86F
:109F800000302368990642BFD9F800300233C9F87F
:109F90000030256815F0060507D104F1190AE368B9
:109FA000D9F800209B1AAB4228DC94F84330226891
:109FB000003318BF012392062DD404F14302394621
:109FC0003046C047013020D02368E568D9F800202A
:109FD00003F00603042B08BFAD1AA36822690CBF67
:109FE00025EAE57500259342C4BF9B1AED184FF092
:109FF00000091A344D451AD1002008E001235246C9
:10A0000039463046C047013003D14FF0FF30BDE83C
:10A01000F0870135C3E7E1185A1C302081F843006E
:10A02000224494F8451082F843100233C5E7012317
:10A03000224639463046C0470130E6D009F10109D1
:10A04000D8E700002DE9F04301F1430C0C46097EEE
:10A0500085B06E291746064698460C9A00F0B380E4
:10A0600022D8632936D00AD8002900F0B9805829AF
:10A0700000F0838004F1420584F8421032E0642944
:10A0800001D06929F6D120681368050603F104019F
:10A090002AD51B681160002B03DA2D225B4284F85D
:10A0A00043206F480A2239E0732900F09D8008D8C8
:10A0B0006F2920D07029DDD1236843F0200323606D
:10A0C00003E0752917D07829D4D1782384F8453056
:10A0D000644855E01368191D1B68116004F14205BE
:10A0E00084F8423001238CE01B68116010F0400FAF
:10A0F00018BF1BB2CFE713682568181D106028062B
:10A1000001D51B6802E06806FBD51B8854486F29FF
:10A1100014BF0A220822002184F843106568A56054
:10A12000002DC0F29580216821F004012160002BF0
:10A130003DD1002D40F08E806546082A0BD1236862
:10A14000DB0708D5236962689A42DEBF302305F831
:10A15000013C05F1FF35ACEB05032361CDF8008030
:10A160003B4603AA21463046FFF7F6FE01304DD1AB
:10A170004FF0FF3005B0BDE8F083394884F8451052
:10A18000136821681D1D1B6815600A060BD5CA07D8
:10A1900044BF41F0200121601BB9226822F0200257
:10A1A00022601022B7E74D0648BF9BB2EFE7654635
:10A1B000B3FBF2F102FB1133C35C05F8013D0B4622
:10A1C0000029F5D1B9E7136825686169181D106089
:10A1D00028061B6801D5196002E06A06FBD51980C4
:10A1E000002323616546B9E71368191D11601D68D6
:10A1F00062680021284600F0ABFC08B1401B60609B
:10A2000063682361002384F84330A7E723692A4663
:10A2100039463046C0470130AAD023689B0713D483
:10A22000E068039B9842B8BF1846A3E701234A465B
:10A2300039463046C04701309AD00135E368039A69
:10A240009B1AAB42F2DCEBE7002504F11909F5E7B4
:10A25000002BACD1037884F8423004F142056CE75E
:10A26000E9C90000FAC9000038B50D4B1C68A36BA2
:10A2700005467BB9182000F04DFC0A4A0A4BA06342
:10A28000C0E90023094B83600B2383810122002353
:10A29000C0E90423A36B00221D615A6138BD00BFD1
:10A2A000500000200E33CDAB34126DE6ECDE05001D
:10A2B00038B5134B1C68A36B7BB9182000F02AFC3F
:10A2C000104A114BA063C0E90023104B83600B239D
:10A2D000838101220023C0E90423A16B0C480A6991
:10A2E0004B690C4C504304FB0300A2FB04230344C2
:10A2F000541C43F10005C1E9044525F0004038BD78
:10A30000500000200E33CDAB34126DE6ECDE0500BC
:10A310002DF451582D7F954C0CB430B5174B0C1EB5
:10A320009DB01D6808DA8B232B604FF0FF301DB005
:10A33000BDE8304002B070474FF40273ADF81430FE
:10A3400014BF04F1FF332346049307934FF6FF73C2
:10A3500002900690ADF81630209A21AB02A928464B
:10A36000019300F06DFD431CBCBF8B232B60002CC0
:10A37000DDD0029B00221A70D9E700BF50000020F8
:10A380000EB400B59CB01DAB029006906FF000417A
:10A39000094807910491094953F8042B0591006875
:10A3A000019302A900F04CFD029B00221A701CB020
:10A3B0005DF804EB03B07047500000200802FFFF77
:10A3C00010B503461A785C1C3AB9013B11F8012B11
:10A3D00003F8012F002AF9D110BD2346F2E7C9B2D4
:10A3E000034610F8012B1AB18A42F9D1184670477A
:10A3F000002918BF0023F9E710F8012B11F8013BE1
:10A40000012A28BF9A42F7D0D01A7047034613F8A2
:10A41000012B002AFBD1181A0138704710B56AB118
:10A420000139841810F8013B11F8012F934203D130
:10A43000A04201D0002BF5D1981A10BD1046FCE7C0
:10A4400070B50139044602B970BD234611F8015FA9
:10A4500003F8015B561E2DB91444A342F4D003F84F
:10A46000015BFAE71C463246EDE7F0B503787BB1B5
:10A47000044623782046661C7BB14A1E631E12F8F0
:10A48000015F4DB113F8017FAF423446F7D0F0E7DA
:10A490000B78002B18BF0020F0BD1846FCE72DE913
:10A4A000F0478046894692461E460F463D4608982C
:10A4B00015F8014B00F0C6FA2044437813F0080366
:10A4C00032D12D2C32D17C78BD1C0122002E5DD0E2
:10A4D000102E09D1302C07D12B7803F0DF03582B35
:10A4E0004FD16C7810260235002A14BF4FF000417E
:10A4F0006FF000410027B1FBF6FC384606FB1C1E3E
:10A50000A4F13003092B17D81C46A64223DD7B1C7F
:10A5100007D084451CD301D1A64519DB00FB0640BA
:10A52000012715F8014BEBE72F46BFE72B2C04BFA3
:10A53000BD1C7C781A46C9E7A4F14103192B01D848
:10A54000373CE2E7A4F16103192B04D8573CDCE760
:10A550004FF0FF37E5E77B1C08D12223C8F8003015
:10A560000846BAF1000F07D1BDE8F08702B14042BA
:10A57000BAF1000FF8D00FB105F1FF39CAF8009019
:10A58000F2E73024002EAFD10826ADE7302CA3D05F
:10A590000A26A9E7084B37B51C68084D236A002B2B
:10A5A00008BF2B46009313460A4601462046FFF794
:10A5B00076FF03B030BD00BF50000020B400002083
:10A5C000F8B50E461446054618B183690BB900F07C
:10A5D000AFF9214B9C422AD16C68A369A360A3897F
:10A5E0001A072ED5236963B323692068C01A6369EB
:10A5F000F6B28342374604DC2146284600F02EF9A5
:10A6000028BBA368013BA36023685A1C22601E700C
:10A6100063690130834204D0A389DB0719D50A2E70
:10A6200017D12146284600F019F990B10FE00B4BE5
:10A630009C4201D1AC68D0E7094B9C4208BFEC6852
:10A64000CBE72146284600F00DF80028CCD04FF08B
:10A65000FF373846F8BD00BF2CCA00004CCA0000C6
:10A660000CCA0000324B70B51D6806460C4625B179
:10A67000AB6913B9284600F05BF92E4B9C420FD111
:10A680006C68B4F90C309AB215072CD4D00611D4EA
:10A690000922326043F04003A3814FF0FF303EE0D7
:10A6A000254B9C4201D1AC68EBE7244B9C4208BF90
:10A6B000EC68E6E7510712D5616B41B104F1440340
:10A6C000994202D0304600F093FA00236363A389D5
:10A6D00023F02403A3810023636023692360A389FB
:10A6E00043F00803A38123694BB9A38903F42073C2
:10A6F000B3F5007F03D02146304600F0CBF9A289A4
:10A7000012F001030CD00023A36063695B42A361D4
:10A71000236953B9B4F90C3013F08000BAD170BD7D
:10A72000920758BF6369A360F2E70020F7E700BF14
:10A73000500000202CCA00004CCA00000CCA0000C7
:10A7400008B5062000F0AAFC012000F0D3FD0000AF
:10A750008A892DE9F041054610070C4658D44B680C
:10A76000002B05DC0B6C002B02DC0020BDE8F08127
:10A77000E66A002EF9D0002312F480522F68216A75
:10A780002B6032D0606DA3895A0705D56368C01A63
:10A79000636B0BB1236CC01A00230246E66A216A80
:10A7A0002846B047431CA38906D129681D2948D8EB
:10A7B000294ACA40D60744D500226260D9042269DA
:10A7C000226004D5421C01D12B6803B96065616B1E
:10A7D0002F600029C9D004F14403994202D02846D1
:10A7E00000F006FA00206063C0E701232846B04766
:10A7F000411CC8D12B68002BC5D01D2B01D0162BB6
:10A8000001D12F60B1E7A38943F04003A381ADE7F5
:10A810000F69002FA9D093070E6808BF4B690F601E
:10A8200018BF0023A6EB07088B60B8F1000F9CDD72
:10A8300043463A46216AA66A2846B047002806DC05
:10A84000A38943F04003A3814FF0FF308EE7074414
:10A85000A8EB0008E9E700BF0100402038B50B690C
:10A8600005460C46DBB118B183690BB900F060F8FE
:10A870000C4B9C4209D16C68B4F90C307BB1214679
:10A880002846BDE83840FFF763BF074B9C4201D123
:10A89000AC68F1E7054B9C4208BFEC68ECE7002090
:10A8A00038BD00BF2CCA00004CCA00000CCA000012
:10A8B000002310B50446C0E90033836081814366FC
:10A8C000C281C0E904338361194608225C30FFF776
:10A8D000FFF9054B6362054BA362054BE362054B31
:10A8E0002462236310BD00BFD5B00000F7B00000A4
:10A8F0002FB1000053B10000014900F085B800BF3E
:10A900005DA8000070B54A1E682555430E4605F146
:10A91000740100F0BBF9044640B10021C0E9001603
:10A920000C30A06005F16802FFF7D2F9204670BD37
:10A93000836910B5044633BBC0E912330365124B7B
:10A94000124A1B688262984204BF0123836100F0AF
:10A950001FF86060204600F01BF8A060204600F061
:10A9600017F80022E06004216068FFF7A1FF0122D0
:10A970000921A068FFF79CFF02221221E068FFF77F
:10A9800097FF0123A36110BDD4C90000F9A80000FE
:10A99000F8B51B4B1E68B369074613B93046FFF77D
:10A9A000C7FF4836D6E90134013B03D5336833B1DC
:10A9B0003668F7E7B4F90C506DB16834F4E7042158
:10A9C0003846FFF79FFF30600028F1D10C233B6031
:10A9D00004462046F8BD0B4B6566C4E90055A560EA
:10A9E000C4E90335C4E905550822294604F15C0091
:10A9F000FFF76EF9C4E90D55C4E91255E9E700BF48
:10AA0000D4C900000100FFFF2DE9F84380468946C4
:10AA100000F14804002614B93046BDE8F883D4E9B3
:10AA20000175013F01D52468F5E7AB89012B07D9F2
:10AA3000B5F90E30013303D029464046C8470643D6
:10AA40006835EEE7D0F8EC00704770B50E46B1F906
:10AA50000E10002996B014461D4607DA00232B601D
:10AA6000B3891A0610D44FF480630EE06A4600F0F2
:10AA7000A3FB0028F2DB019A02F47042A2F5005316
:10AA80005A425A412A60EEE740230020236016B064
:10AA900070BD00008B8973B59D0706460C4607D52F
:10AAA00004F14703236023610123636102B070BD99
:10AAB00001AB6A46FFF7C9FF00990546304600F032
:10AAC000E5F848B9B4F90C309A05EFD423F0030344
:10AAD00043F00203A381E3E70D4BB362A389206037
:10AAE00043F08003A381009B6361019B20615BB104
:10AAF000B4F90E10304600F071FB28B1A38923F0A1
:10AB0000030343F00103A381A3891D43A581CDE77E
:10AB1000F9A80000024B0146186800F0B7B800BF62
:10AB20005000002082B001B901A942B14BB11378A5
:10AB30000B601278101C18BF012002B0704710463D
:10AB4000FBE76FF00100F8E70000000000000000E4
:10AB500001F0FF01102A2BDB10F0070F08D010F8CE
:10AB6000013B013A8B422DD010F0070F42B3F6D1D2
:10AB7000F0B441EA012141EA014122F007047FF0EB
:10AB800000070023F0E80256083C85EA010586EA42
:10AB9000010685FA47F5A3FA87F586FA47F6A5FA7E
:10ABA00087F68EB9EED1F0BC01F0FF0102F007028A
:10ABB00032B110F8013B013A83EA010313B1F8D135
:10ABC0000020704701387047002D06BF3546033816
:10ABD000073815F0010F07D1013015F4807F02BF4F
:10ABE000013015F4C03F0130F0BC0138704700BFA0
:10ABF00038B50546002945D051F8043C0C1F002B00
:10AC0000B8BFE41800F00CFB1F4A1368104633B9B4
:10AC1000636014602846BDE8384000F002BBA342E0
:10AC20000CD921686218934204BF1A685B6863609C
:10AC300004BF521822600460ECE713465A680AB158
:10AC4000A242FAD919685818A0420BD120680144D1
:10AC5000581882421960DDD1106852685A60014468
:10AC60001960D7E702D90C232B60D3E7206821189D
:10AC70008A4204BF11685268626004BF09182160EB
:10AC80005C60C7E738BD00BF607A012070B5CD1C9D
:10AC900025F0030508350C2D38BF0C25002D064680
:10ACA00001DBA94203D90C233360002070BD00F002
:10ACB000B7FA214A1468214691B9204C23681BB980
:10ACC000304600F0B3F920602946304600F0AEF976
:10ACD000431C24D10C233360304600F0A2FAE4E791
:10ACE0000B685B1B18D40B2B0FD90B60CD50CC1805
:10ACF000304600F096FA04F10B00231D20F0070007
:10AD0000C31AD3D05A42E250D0E78C424B6816BFE8
:10AD1000636013600C46EBE70C464968CCE7C41C43
:10AD200024F00304A04205D0211A304600F07EF939
:10AD30000130CFD02560DBE7607A0120647A012002
:10AD4000F8B5074614460E4621B91146BDE8F8404D
:10AD5000FFF79CBF22B9FFF74BFF25462846F8BDF9
:10AD600000F060FAA0420FD221463846FFF78EFF6E
:10AD700005460028F2D031462246FEF785FF3146CF
:10AD80003846FFF735FFE9E73546E7E72DE9F047B5
:10AD90008E689E4282460C469046994637D88A89EC
:10ADA00012F4906F31D0256809696F1A6569022322
:10ADB00005EB450595FBF3F509F101033B449D4285
:10ADC00038BF1D46530530D52946FFF75FFF0646BD
:10ADD00050B90C23CAF80030A38943F04003A38183
:10ADE0004FF0FF30BDE8F0873A462169FEF74CFF8F
:10ADF000A38923F4906343F08003A38126616561F6
:10AE00003E44ED1B2660A5604E464E4500D94E4699
:10AE1000324641462068FEF742FFA3689B1BA360B1
:10AE200023681E4426600020DCE72A46FFF788FFDF
:10AE300006460028E2D121695046FFF7D9FEC8E74F
:10AE40002DE9F04F9DB0804603938B891D060C467B
:10AE500016460FD50B696BB94021FFF717FF20602D
:10AE6000206128B90C23C8F800304FF0FF30C7E04C
:10AE7000402363610023099320238DF82930302378
:10AE80008DF82A304FF0010B37463D4615F8013B4F
:10AE90000BB1252B3ED1B7EB060A0BD053463246F9
:10AEA00021464046FFF772FF013000F0A480099B65
:10AEB000534409933B78002B00F09D8000234FF012
:10AEC000FF32CDE90523049307938DF853301A938D
:10AED0002F46052217F8011B4F48FFF739FE049B48
:10AEE000D0B9D90644BF20228DF853201A0744BF99
:10AEF0002B228DF853202A782A2A15D0079A2F461C
:10AF000000200A25394611F8013B303B092B4DD969
:10AF1000B8B10FE02F46B8E73F4A801A0BFA00F0AD
:10AF2000184304903D46D3E7039A111D126803911C
:10AF3000002A01DB079204E0524243F00203079229
:10AF400004933B782E2B0CD17B782A2B33D1039B97
:10AF50001A1D1B680392002BB8BF4FF0FF33023756
:10AF600005932E4D397803222846FFF7F1FD38B1BD
:10AF70004023401B03FA00F0049B03430137049372
:10AF8000397827488DF8281006227E1CFFF7E0FD4F
:10AF9000002838D0234B13BB039B073323F0070350
:10AFA00008330393099B4B4409936DE705FB023279
:10AFB00001200F46A6E700230137059319460A250D
:10AFC000384610F8012B303A092A03D9002BC8D093
:10AFD0000591C6E705FB012101230746F0E703AB16
:10AFE00000932246104B04A94046AFF30080B0F115
:10AFF000FF3F8146D6D1A3895B063FF536AF09985E
:10B000001DB0BDE8F08F03AB00932246064B04A9A8
:10B010004046FFF717F8EAE7D8C90000DEC900008C
:10B02000E2C90000000000008DAD000038B5064CFC
:10B03000002305460846236000F046F9431C02D170
:10B04000236803B12B6038BDF48D01201F2938B56A
:10B0500004460D4604D9162303604FF0FF3038BD77
:10B06000426C12B152F821304BB9204600F030F852
:10B070002A4601462046BDE8384000F017B8012BAB
:10B080000AD0591C03D1162303600120E7E70024EE
:10B0900042F82540284698470020E0E7024B014649
:10B0A0001868FFF7D3BF00BF5000002038B5074C29
:10B0B0000023054608461146236000F0EDF8431CC6
:10B0C00002D1236803B12B6038BD00BFF48D01208D
:10B0D00000F0D2B810B50C46B1F90E1000F0AAF885
:10B0E0000028ABBF636DA3891B1823F48053ACBF4A
:10B0F0006365A38110BD2DE9F0411F468B89DB05F7
:10B1000005460C46164605D502230022B1F90E105D
:10B1100000F074F8A389B4F90E1023F48053A381CE
:10B1200032463B462846BDE8F04100F023B810B552
:10B130000C46B1F90E1000F061F8431CA38915BF4D
:10B14000606523F4805343F48053A38118BFA38127
:10B1500010BDB1F90E1000F01FB849B1FF2A85BF2C
:10B160008A2303600A704FF0FF3098BF01207047B8
:10B170000846704738B5074C054608461146002278
:10B1800022601A4600F0AEF8431C02D1236803B1D6
:10B190002B6038BDF48D012038B5064C00230546E0
:10B1A0000846236000F058F8431C02D1236803B11D
:10B1B0002B6038BDF48D012038B5074C00230546BF
:10B1C00008461146236000F04FF8431C02D1236863
:10B1D00003B12B6038BD00BFF48D012038B5064C9B
:10B1E000002305460846236000F04EF8431C02D1B8
:10B1F000236803B12B6038BDF48D012038B5074CAE
:10B20000054608461146002222601A4600F04CF816
:10B21000431C02D1236803B12B6038BDF48D01209B
:10B220007047704751F8043C181F002BBCBF0B58E7
:10B23000C018704738B5074C05460846114600222D
:10B2400022601A4600F038F8431C02D1236803B18B
:10B250002B6038BDF48D0120024B58221A604FF04C
:10B26000FF307047F48D0120024B58221A604FF0D6
:10B27000FF307047F48D0120024B58221A604FF0C6
:10B28000FF307047F48D0120024B58221A600020D5
:10B29000704700BFF48D0120024B58221A604FF016
:10B2A000FF307047F48D0120024B58221A604FF096
:10B2B000FF307047F48D0120024B58221A604FF086
:10B2C000FF307047F48D0120044A05491368002BB4
:10B2D00008BF0B461844106018467047687A012072
:10B2E000F88D0120024B58221A604FF0FF30704752
:10B2F000F48D0120FEE700BFF8B500BFF8BC08BC24
:10B300009E467047F8B500BFF8BC08BC9E46704723
:10B31000646174610000000094B300001D0500002A
:10B320009DB300000D060000A5B30000D90B00007E
:10B33000ACB30000E90C0000B1B30000330800001A
:10B34000BCB3000077060000C1B30000250F000069
:10B35000CDB300004F050000D7B30000F10A000094
:10B36000E5B30000BF090000F2B30000FB070000D6
:10B3700072616E646F6D00616C6C006C617374005F
:10B3800066616C7365007472756500252E313573C6
:10B390002E2E2E006D616B654C69737400616464C0
:10B3A0004C6173740064656C657465006A6F696EE6
:10B3B00000636F707946726F6D546F0066696E64DA
:10B3C000006A6F696E537472696E677300756E6997
:10B3D000636F6465417400756E69636F646553746F
:10B3E00072696E67006E6577427974654172726149
:10B3F0007900667265654D656D6F727900000000B9
:10B4000065B400007D1300006AB4000097130000CB
:10B41000A5B300009B13000070B40000811300006E
:10B420007AB400009F13000083B40000A31300004F
:10B430008DB40000A713000098B40000AB13000007
:10B44000A4B4000085130000ADB400008F13000009
:10B45000B7B4000089130000C2B4000093130000C9
:10B4600066696C65006F70656E00636C6F73650074
:10B47000656E644F6646696C6500726561644C690F
:10B480006E65007265616442797465730061707005
:10B49000656E644C696E6500617070656E644279BA
:10B4A0007465730066696C6553697A6500737461CD
:10B4B00072744C697374006E657874496E4C69736C
:10B4C000740073797374656D496E666F00000000D7
:10B4D000D0150000E0150000F4150000681600000B
:10B4E0009A160000CA160000FC1600001E17000085
:10B4F0005A17000092170000E217000022180000FF
:10B500008A180000C8180000E81800001C19000084
:10B510005C1900007E190000A8190000D219000073
:10B52000121A00008A1A0000481B0000BA1B000013
:10B53000041C0000681C0000841C0000A21C000009
:10B540003C1D0000781D0000E81D0000161E0000D4
:10B550003E1E0000761E0000DA1E00003E1F0000A6
:10B56000821F0000C61F000036200000A620000039
:10B57000F0200000342100006A210000AE2100000C
:10B58000F42100003A2200008C220000E222000098
:10B590002023000094230000C82300000E24000094
:10B5A000542400009A240000D42400001A2500002E
:10B5B00060250000BC260000A81900001C1900002E
:10B5C000D4250000D0150000082600002E2600001B
:10B5D0006226000088260000D0150000D01500006B
:10B5E000D0150000D015000032270000722700009F
:10B5F000B62700000A280000302800007E2800003E
:10B60000A4280000D4280000D0150000D0150000A8
:10B61000F228000024290000562900008A29000091
:10B62000AE290000E2290000302A0000522A000062
:10B63000742A0000A62A0000D82A0000FC2A000074
:10B64000202B0000522B0000762B0000D0150000AC
:10B65000D0150000D0150000D0150000D015000056
:10B66000A82B0000CE2B0000F42B00001A2C0000A9
:10B67000402C0000742C0000A82C0000DC2C0000E2
:10B68000102D0000362D00005C2D0000902D0000D4
:10B69000D0150000D0150000D0150000D015000016
:10B6A000D0150000D0150000D0150000D015000006
:10B6B000D0150000D0150000D0150000D0150000F6
:10B6C000D0150000D0150000B62D0000E62D0000BA
:10B6D0005B2564206974656D206C6973745D002856
:10B6E00025642062797465732900286F626A656336
:10B6F0007420747970653A2025642900537461635D
:10B700006B20756E646572666C6F7700626F6F6C2C
:10B7100065616E006E756D62657200737472696E3C
:10B7200067006C697374006279746520617272617C
:10B7300079000000070000000300000095B700003A
:10B74000012F00009DB70000AD2F0000A6B700003C
:10B750004B300000AFB70000052F0000B8B7000065
:10B760004F300000C0B700003D3000000000000076
:10B7700001000000020000000300000004000000BF
:10B780000A0000001D0000006D6963726F3A626973
:10B790007420763200686173546F6E6500706C615E
:10B7A00079546F6E6500686173536572766F0073CC
:10B7B0006574536572766F00646163496E697400E5
:10B7C000646163577269746500474320746F6F6BDF
:10B7D0002025642075736563733B20667265652060
:10B7E000256420776F726473003C496E74656765E9
:10B7F000723E003C4C6973743E003C4F626A656364
:10B80000743E003C4279746541727261793E000D6C
:10B810000A564D2050616E69633A2025730D0A0067
:10B820006D697363000000005DB80000853D000095
:10B8300066B80000093D00006AB80000553C0000F1
:10B8400072B80000F73B00007CB80000893B0000A4
:10B8500088B800008B3A00006E756C6C00686578E3
:10B86000546F496E740073696E006A736F6E47653A
:10B8700074006A736F6E436F756E74006A736F6ED7
:10B8800056616C75654174006A736F6E4B657941E2
:10B8900074000000F0B80000E53D0000F8B80000BA
:10B8A000E93D000002B90000FB3D00000BB90000BB
:10B8B000013E000016B90000073E000022B900005A
:10B8C0000D3E000037B90000133E00004CB90000E7
:10B8D000193E000058B900001F3E000068B9000082
:10B8E000EF3D000074B90000F53D00006E65740086
:10B8F0006861735769466900737461727457694669
:10B90000690073746F705769466900776966695397
:10B910007461747573006D79495041646472657324
:10B9200073006874747053657276657247657452FB
:10B9300065717565737400726573706F6E64546FB2
:10B9400048747470526571756573740068747470AE
:10B95000436F6E6E65637400687474704973436FEF
:10B960006E6E656374656400687474705265717599
:10B970006573740068747470526573706F6E73656C
:10B980000000000004000000030000000A000000A6
:10B990000700000006000000000000000008080882
:10B9A00000080A4A4000000A5FEA5FEA0ED92ED377
:10B9B0006E19324489330C924C924D0808000000F5
:10B9C00004880808040804848488000A448A400023
:10B9D000048EC480000000048800000EC000000037
:10B9E00000080001224488100C9252524C048C84AE
:10B9F000848E1C824C901E1EC244924C06CA525F1A
:10BA0000E21FF01EC13E02448ED12E1FE244881078
:10BA10000ED12ED12E0ED12EC488000800080000B1
:10BA2000048004880244880482000EC00EC008040A
:10BA30008244880ED126C0040ED135B36C0C925EC0
:10BA4000D2521C925C925C0ED010100E1C9252527C
:10BA50005C1ED01C901E1ED01C90100ED013712E98
:10BA600012525ED2521C8808081C1FE242524C122D
:10BA700054981492101010101E113B75B1311139E9
:10BA800035B3710C9252524C1C925C90100C925235
:10BA90004C861C925C92510ED00C825C1FE4848414
:10BAA00084125252524C1131312A44113135BB713A
:10BAB00012524C9252112A4484841EC488101E0EC5
:10BAC000C808080E10080482410EC242424E048A81
:10BAD000400000000000001F0804800000000ED29B
:10BAE000524F10101C925C000ED0100E02424ED22B
:10BAF0004E0C925C900E06C81C88080ED24EC24CAA
:10BB000010101C92520800080808024002424C1013
:10BB1000149814920808080806001B75B131001C1F
:10BB2000925252000C92524C001C925C90000ED229
:10BB30004EC2000ED010100006C8049808080EC8A7
:10BB400007001252524F0011312A4400113135BB07
:10BB500000124C8C9200112A4498001EC4881E06C4
:10BB6000C48C8486080808080818080C8818000087
:10BB70000C836000000000000100000002000000D3
:10BB800003000000040000000500000006000000A3
:10BB90000700000008000000090000000A00000083
:10BBA0000B0000000C0000000D0000000E00000063
:10BBB0000F00000010000000120000001400000040
:10BBC00016000000180000001A0000001C00000011
:10BBD0001E000000200000002300000026000000DE
:10BBE000290000002C0000002F000000320000009F
:10BBF000360000003A0000003E0000004200000055
:10BC0000460000004B0000005000000055000000FE
:10BC10005A00000061000000680000006F00000092
:10BC2000760000007D000000840000008B00000012
:10BC30009200000099000000A0000000A700000092
:10BC4000AE000000B5000000BC000000C300000012
:10BC5000CA000000D1000000D8000000DF00000092
:10BC6000E6000000ED000000F4000000FB00000012
:10BC7000FF000000000000000200000004000000BF
:10BC80000100000003000000ECBC0000393E000091
:10BC9000F7BC0000A942000001BD0000F53E000015
:10BCA0000EBD00001541000015BD000061410000FF
:10BCB0001EBD0000B14100002ABD0000A5400000EB
:10BCC0003BBD0000493F000048BD00002D40000082
:10BCD000150000001600000017000000180000000A
:10BCE00019000000646973706C6179006C696768A1
:10BCF000744C6576656C006D62446973706C617933
:10BD0000006D62446973706C61794F6666006D62A4
:10BD1000506C6F74006D62556E706C6F74006D6264
:10BD2000447261775368617065006D625368617039
:10BD300065466F724C6574746572006E656F50690C
:10BD400078656C53656E64006E656F506978656CDC
:10BD500053657450696E004E6F7420656E6F756721
:10BD60006820726F6F6D206576656E206166746500
:10BD70007220636F6D70616374696F6E00436F6DE5
:10BD800070616374656420466C61736820636F64DE
:10BD9000652073746F72650A256420627974657317
:10BDA000207573656420282564252529206F662069
:10BDB000256400426164207265636F726420666F5F
:10BDC000756E6420647572696E6720696E69746946
:10BDD000616C697A6174696F6E0025642025642046
:10BDE00025642028256420776F72647329002564F8
:10BDF000207265636F7264732C20256420776F72E4
:10BE000064732C206D617849442025642C20636F75
:10BE10006D70616374696F6E206379636C65732004
:10BE2000256400526573746F726564202564207305
:10BE30006372697074730053746172746564007224
:10BE40006164696F00000000D8BE0000994B0000DB
:10BE5000E5BE00000D4E0000F5BE0000A14D000043
:10BE600003BF00006D4F00000EBF0000C14B00007B
:10BE70001EBF0000514C000032BF0000354C0000D6
:10BE800041BF0000495100004DBF0000C5500000F7
:10BE900056BF00006950000061BF0000B94F0000AC
:10BEA0006CBF0000F14F000075BF00002150000082
:10BEB0007EBF0000D14B00008DBF0000B14B0000E1
:10BEC00096BF0000E14B00006E6F6E65006F7468F6
:10BED000657200706169720064697361626C6552B9
:10BEE0006164696F006D6573736167655265636551
:10BEF00069766564007061636B657452656365693A
:10BF00007665007061636B657453656E640072657D
:10BF1000636569766564496E74656765720072650C
:10BF20006365697665644D6573736167655479709F
:10BF300065007265636569766564537472696E67DE
:10BF40000073656E64496E74656765720073656E33
:10BF500064506169720073656E64537472696E67D0
:10BF6000007365744368616E6E656C007365744739
:10BF7000726F757000736574506F776572007369C6
:10BF8000676E616C537472656E6774680064657681
:10BF90006963654944006C6173744D6573736167CF
:10BFA00065494400556E6B6E6F776E207072696DD7
:10BFB0006974697665205B25733A25735D0000001E
:10BFC00000000000963007772C610EEEBA510999F7
:10BFD00019C46D078FF46A7035A563E9A395649E53
:10BFE0003288DB0EA4B8DC791EE9D5E088D9D29777
:10BFF0002B4CB609BD7CB17E072DB8E7911DBF90D3
:10C000006410B71DF220B06A4871B9F3DE41BE84F6
:10C010007DD4DA1AEBE4DD6D51B5D4F4C785D38352
:10C0200056986C13C0A86B647AF962FDECC9658AF6
:10C030004F5C0114D96C0663633D0FFAF50D088D52
:10C04000C8206E3B5E10694CE44160D5727167A2F6
:10C05000D1E4033C47D4044BFD850DD26BB50AA552
:10C06000FAA8B5356C98B242D6C9BBDB40F9BCAC76
:10C07000E36CD832755CDF45CF0DD6DC593DD1ABD2
:10C08000AC30D9263A00DE518051D7C81661D0BFF6
:10C09000B5F4B42123C4B3569995BACF0FA5BDB852
:10C0A0009EB802280888055FB2D90CC624E90BB1F6
:10C0B000877C6F2F114C6858AB1D61C13D2D66B652
:10C0C0009041DC760671DB01BC20D2982A10D5EFB6
:10C0D0008985B1711FB5B606A5E4BF9F33D4B8E812
:10C0E000A2C9077834F9000F8EA8099618980EE1B6
:10C0F000BB0D6A7F2D3D6D08976C6491015C63E612
:10C10000F4516B6B62616C1CD83065854E0062F235
:10C11000ED95066C7BA5011BC1F4088257C40FF591
:10C12000C6D9B06550E9B712EAB8BE8B7C88B9FCB5
:10C13000DF1DDD62492DDA15F37CD38C654CD4FB11
:10C140005861B24DCE51B53A7400BCA3E230BBD4B5
:10C1500041A5DF4AD795D83D6DC4D1A4FBF4D6D311
:10C160006AE96943FCD96E34468867ADD0B860DAB5
:10C17000732D0444E51D03335F4C0AAAC97C0DDD11
:10C180003C710550AA41022710100BBE86200CC935
:10C1900025B56857B3856F2009D466B99FE461CE91
:10C1A0000EF9DE5E98C9D9292298D0B0B4A8D7C7B5
:10C1B000173DB359810DB42E3B5CBDB7AD6CBAC011
:10C1C0002083B8EDB6B3BF9A0CE2B6039AD2B1742D
:10C1D0003947D5EAAF77D29D1526DB048316DC7389
:10C1E000120B63E3843B64943E6A6D0DA85A6A7A2D
:10C1F0000BCF0EE49DFF099327AE000AB19E077D89
:10C2000044930FF0D2A3088768F2011EFEC20669AC
:10C210005D5762F7CB67658071366C19E7066B6E08
:10C22000761BD4FEE02BD3895A7ADA10CC4ADD672C
:10C230006FDFB9F9F9EFBE8E43BEB717D58EB06088
:10C24000E8A3D6D67E93D1A1C4C2D83852F2DF4F2C
:10C25000F167BBD16757BCA6DD06B53F4B36B24888
:10C26000DA2B0DD84C1B0AAFF64A0336607A04412C
:10C27000C3EF60DF55DF67A8EF8E6E3179BE694688
:10C280008CB361CB1A8366BCA0D26F2536E26852AC
:10C2900095770CCC03470BBBB91602222F26055508
:10C2A000BE3BBAC5280BBDB2925AB42B046AB35C2C
:10C2B000A7FFD7C231CFD0B58B9ED92C1DAEDE5B88
:10C2C000B0C2649B26F263EC9CA36A750A936D026C
:10C2D000A906099C3F360EEB8567077213570005C8
:10C2E000824ABF95147AB8E2AE2BB17B381BB60CEC
:10C2F0009B8ED2920DBED5E5B7EFDC7C21DFDB0B48
:10C30000D4D2D38642E2D4F1F8B3DD686E83DA1F6B
:10C31000CD16BE815B26B9F6E177B06F7747B718C7
:10C32000E65A0888706A0FFFCA3B06665C0B01116B
:10C33000FF9E658F69AE62F8D3FF6B6145CF6C16C7
:10C3400078E20AA0EED20DD75483044EC2B303396B
:10C35000612667A7F71660D04D476949DB776E3EC7
:10C360004A6AD1AEDC5AD6D9660BDF40F03BD837EB
:10C3700053AEBCA9C59EBBDE7FCFB247E9FFB53047
:10C380001CF2BDBD8AC2BACA3093B353A6A3B4246B
:10C390000536D0BA9306D7CD2957DE54BF67D923C7
:10C3A0002E7A66B3B84A61C4021B685D942B6F2A6B
:10C3B00037BE0BB4A18E0CC31BDF055A8DEF022DC7
:10C3C000416C6C207461736B732073746F70706553
:10C3D00064007631303600202573202573004D65CA
:10C3E0006D6F727920636C6561726564004E6F20B9
:10C3F00066726565207461736B20656E7472696521
:10C40000730000005CC400007966000069C400008D
:10C41000F560000075C40000496600007BC40000A0
:10C420005966000081C400006966000087C40000EE
:10C430002561000091C40000C166000099C400009D
:10C4400015640000A2C40000AD610000AAC4000091
:10C450004563000073656E736F727300616363659B
:10C460006C65726174696F6E0074656D7065726180
:10C47000747572650074696C74580074696C7459D1
:10C480000074696C745A00746F75636852656164F6
:10C49000006932635265616400693263577269747E
:10C4A000650072656164444854006D6963726F7021
:10C4B000686F6E65000000002CC500004167000039
:10C4C0003AC500004567000043C500005167000001
:10C4D0004DC500005567000056C5000059670000B3
:10C4E0005BC500005D67000060C50000616700007B
:10C4F0006CC500006567000073C500006967000037
:10C500007CC500006D67000081C5000071670000F8
:10C510008CC500007567000096C5000049670000E3
:10C52000A0C500004D67000074667400656E61620E
:10C530006C65446973706C617900676574576964F0
:10C54000746800676574486569676874007365742A
:10C55000506978656C006C696E6500726563740083
:10C56000726F756E646564526563740063697263AB
:10C570006C6500747269616E676C650074657874CF
:10C5800000746674546F75636865640074667454EF
:10C590006F7563685800746674546F7563685900EA
:10C5A000746674546F7563685072657373757265E1
:10C5B0000076617273000000D8C50000D96B0000DE
:10C5C000E2C50000B96B0000EBC50000956B0000F0
:10C5D000F7C50000276B00007661724578697374B7
:10C5E00073007661724E616D6564007365745661A7
:10C5F000724E616D6564007661724E616D65466F65
:10C6000072496E6465780057656C636F6D65207460
:10C610006F204D6963726F426C6F636B73210070A2
:10C620005F73706920213D204E554C4C002F686F80
:10C630006D652F6769742F2E706C6174666F726DF3
:10C64000696F2F7061636B616765732F6672616DCF
:10C6500065776F726B2D61726475696E6F6E6F7244
:10C660006469636E7266352F6C69627261726965A6
:10C67000732F5350492F5350492E637070005350FD
:10C6800049436C6173733A3A535049436C61737315
:10C69000284E52465F5350495F547970652A2C20CA
:10C6A00075696E74385F742C2075696E74385F74A8
:10C6B0002C2075696E74385F74290000000000003A
:10C6C00000000000D96D0000916D0000C76D0000F2
:10C6D000CD6D0000D36D0000C56D000002000000AC
:10C6E00003000000040000001F0000001C00000008
:10C6F0000E000000250000000B0000000A000000F2
:10C70000090000001E000000170000000C000000DF
:10C7100011000000010000000D00000022000000D8
:10C72000FFFFFFFFFFFFFFFF1A00000020000000D7
:10C7300015000000160000000F00000018000000A7
:10C74000130000002400000000000000140000009E
:10C7500005000000100000000800000019000000A3
:10C76000060000002800000000000000000000009B
:10C770009F740000857B0000157500002175000086
:10C780001B7500009D740000957400002975000061
:10C79000B97400009174000000C001400010024014
:10C7A00000200240000000000000000000003043B4
:10C7B00000000000000030C37371727400000000BC
:10C7C000FB21F93FFB2109407CD91240FB21194094
:10C7D0007A6A1F407CD92240BBFD2540FB212940BD
:10C7E0003A462C407A6A2F405C4731407CD932402F
:10C7F0009C6B3440BBFD3540DB8F3740FB2139401B
:10C800001BB43A403A463C405AD83D407A6A3F40D1
:10C810004C7E40405C4741406C1042407CD94240D5
:10C820008CA243409C6B4440AC344540BBFD45402A
:10C83000CBC64640DB8F4740EB584840FB21494080
:10C8400083F9A200444E6E00FC291500D157270041
:10C85000DD34F50062DBC0003C9995004190430057
:10C860006351FE00BBDEAB00B761C5003A6E240029
:10C87000D24D42004906E00009EA2E001C92D10088
:10C88000EB1DFE0029B11C00E83EA700F535820033
:10C8900044BB2E009CE98400B4267000417E5F00FA
:10C8A000D6913900538339009CF439008B5F8400A2
:10C8B00028F9BD00F81F3B00DEFF97000F98050028
:10C8C000112FEF000A5A8B006D1F6D00CF7E3600CE
:10C8D00009CB2700464FB7009E663F002DEA5F0058
:10C8E000BA277500E5EBC7003D7BF100F73907007B
:10C8F00092528A00FB6BEA001FB15F00085D8D0059
:10C90000300356007BFC4600F0AB6B0020BCCF0030
:10C9100036F49A00E3A91D005E619100081BE60051
:10C9200085996500A0145F008D40680080D8FF00E5
:10C9300027734D0006063100CA561500C9A87300BA
:10C940007BE260006B8CC00000000040FB21F93FDF
:10C95000000000002D44743E000000809846F83C22
:10C960000000006051CC783B00000080831BF03950
:10C970000000004020257A38000000802282E33643
:10C98000000000001DF369350200000003000000F4
:10C9900004000000060000002C2066756E637469B8
:10C9A0006F6E3A2000617373657274696F6E202236
:10C9B000257322206661696C65643A2066696C653E
:10C9C00020222573222C206C696E65202564257336
:10C9D00025730A0054000020232D302B2000686CA2
:10C9E0004C00656667454647003031323334353692
:10C9F00037383941424344454600303132333435CB
:10CA000036373839616263646566000000000000F3
:10CA10000000000000000000000000000000000016
:10CA20000000000000000000000000000000000006
:10CA300000000000000000000000000000000000F6
:10CA400000000000000000000000000000000000E6
:10CA500000000000000000000000000000000000D6
:10CA60000000000000000000000000004300504FE4
:10CA70005349580000202020202020202020282852
:10CA8000282828202020202020202020202020208E
:10CA900020202020208810101010101010101010CE
:10CAA00010101010100404040404040404040410FE
:10CAB000101010101010414141414141010101018C
:10CAC0000101010101010101010101010101010156
:10CAD0001010101010104242424242420202020262
:10CAE0000202020202020202020202020202020226
:10CAF00010101010200000000000000000000000D6
:10CB00000000000000000000000000000000000025
:10CB10000000000000000000000000000000000015
:10CB20000000000000000000000000000000000005
:10CB300000000000000000000000000000000000F5
:10CB400000000000000000000000000000000000E5
:10CB500000000000000000000000000000000000D5
:10CB600000000000000000000000000000000000C5
:0CCB7000000000000000000000000000B9
:08CB7C00C438FF7F0100000036
:10CB8400FFFFFFFFD007000001000000E803DC0501
:10CB9400DC05DC05DC050000FFFFFFFFFFFFFFFFF6
:10CBA4001800000019FCFFFFFFFFFFFFFF0000005B
:10CBB4000090D003FFFFFFFFFFFFFFFFFFFFFFFF1A
:10CBC4000A0000000100000008000000010000004D
:10CBD40054000020000000002CCA00004CCA0000D1
:10CBE4000CCA00000000000000000000000000006B
:10CBF4000000000000000000000000000000000031
:10CC04000000000000000000000000000000000020
:10CC14000000000000000000000000000000000010
:10CC24000000000000000000000000000000000000
:10CC340000000000430000000000000000000000AD
:10CC440000000000000000000000000000000000E0
:10CC5400000000004300000000000000000000008D
:10CC640000000000000000000000000000000000C0
:10CC7400000000004300000000000000000000006D
:10CC840000000000000000000000000000000000A0
:10CC9400000000004300000000000000000000004D
:10CCA4000000000000000000000000000000000080
:10CCB400000000004300000000000000000000002D
:10CCC4000000000000000000000000000000000060
:10CCD400000000004300000000000000000000000D
:10CCE4000000000000000000000000000000000040
:10CCF40000000000430000000000000000000000ED
:10CD0400000000000000000000000000000000001F
:10CD1400000000005BB1000025AB00000000000033
:10CD240074CA000092B300001FB800001FB80000CE
:10CD34001FB800001FB800001FB800001FB8000093
:10CD44001FB800001FB800001FB80000FFFFFFFF5E
:10CD5400FFFFFFFFFFFFFFFFFFFF00000100415344
:10CD640043494900000000000000000000000000EA
:10CD7400000000000000000000000000000041531B
:10CD840043494900000000000000000000000000CA
:10CD9400000000000000000000000000000000008F
:10CDA400250400005D6D0000B971000029770000C2
:04CDB4000104000076
:040000030000727512
:00000001FF
